:100000000270940271B80000000000026D850000CB
:100010000000000271DF000000000032000000005C
:100020000000000241AA0000000000026E930000E0
:1000300074A21200C4E81200FFE91200FF12013698
:100040002274A21200C4E81200FFE71200FF09D5D3
:1000500082F81201362274A21200C4E81200FF7462
:10006000A31200C412011FF709D58204120136221F
:10007000C296D297000000C29780E974A21200C411
:10008000E81200FF1200882274A31200C412011F9C
:10009000F91201362274A27A08C296000000C297B3
:1000A000335005D2960200AAC296D297000000C231
:1000B00097DAEDD29600D297000000309604C297EE
:1000C000C322D3227A08D296D29700000000000003
:1000D00000000000000000000000C296000000C206
:1000E00097335005D2960200EBC296D297000000DB
:1000F000C297DAEDD29600D297000000C297227A1A
:1001000008335005D29602010BC296D29700000028
:10011000C297DAEDD29600D297000000C297227AF9
:1001200008D296C29700000000D297C3309601B360
:1001300033DAF0C29722C296000000D29700000086
:10014000D29622787C76000876007880E6543FF6D6
:100150007800797CC082758207120041D082120536
:10016000DB227802797EC082758205120056D08229
:10017000227882E603C4540775F018A4C0E07880A2
:10018000E6C4540375F00AA4F5F0E6540F25F0D048
:10019000F025F075F03CA4C0F0C0E0787FE6C454D0
:1001A0000775F00AA4F5F0E6540F25F0D0F025F01D
:1001B000F5F0D0E03400C5F02250523430322076D1
:1001C00065722E3132352E32204864773A48203419
:1001D000303030752031342D31312D3034203132F2
:1001E0003A34392020284329526F676572205370B2
:1001F0002E4A2E207777772E726F6765722E706C7D
:100200002C2074656C2F666178202B3438203535AE
:100210002032373230313332202843296A502D7052
:100220006C2C204D6F6E61204C6973612043452C0E
:100230002049534F393030312C2031737420436CB6
:10024000617373D320202052204520532045205431
:10025000D25052333032204C434420763132352E46
:1002600032004350523A20004C6F633A20004C4F0A
:10027000433A2000D22020202020202020202020AF
:100280002020202020D200454E545259202020000A
:1002900045584954202020200044555459204558A1
:1002A000495400494E5445524E414C0020202020D4
:1002B000200020D1466C6173682043524320457270
:1002C000726F722000D32053657276696365204F88
:1002D0004E00D32053657276696365204F46460011
:1002E000D2204D4153544552204944203D20203FC7
:1002F0002000D32020202055205320452052D220FA
:100300002050726F6772616D6D696E6700D2202038
:100310002020202020202020202020202020D2D576
:1003200001055245473A200000D3D5021044206F02
:100330002077206E206C206F206120642000D12067
:1003400020202020202020202020202020202020AD
:10035000D1D5030C50617373776F72643F203A20DC
:1003600000D2D50410204163636573732064656E09
:10037000696564202000D2D5051020416363657350
:1003800073206772616E7465642000D1D5041020FB
:100390004163636573732064656E6965642020D270
:1003A000D50610204E6F204475616C20456E747226
:1003B00079202000D3D509104475616C20456E74F6
:1003C0007279204D6F64652000D1D50A0A20202063
:1003D0004572726F722023002020202000D1D50C9E
:1003E0001020202041504220526573657420202047
:1003F0002000D2D50E104C696D6974206578636554
:1004000065646564202000D50F0C4E4F524D414C61
:1004100020202020202000D1D5041020204143435B
:100420004553532044454E59202020D2D51010204A
:100430004150422056696F6C6174696F6E202000D4
:10044000D1D50D10202020204964656E74204F4BBB
:1004500020202020D2D51010204150422056696F14
:100460006C6174696F6E202000D2D51110204E6F20
:10047000206F6E6520696E73696465202000D1D598
:1004800012102020456E746572204944203D203FA3
:10049000202000D1D5041020204143434553532050
:1004A00044454E59202020D2D506102020496E7098
:1004B000757420426C6F636B73202000D1D50410DB
:1004C00020204143434553532044454E592020208A
:1004D000D2D507102020434C4F534544204D4F4464
:1004E0004520202000D1D50410202041434345530E
:1004F000532044454E59202020D2D508104F757402
:10050000206F662074696D65207A6F6E6500D1D5A5
:10051000041020204143434553532044454E592065
:100520002020D2D50B10204F464620636F6E6469A1
:1005300074696F6E202000D1D513102020535749C5
:100540005443482044454E59202020D2D508104F0E
:100550007574206F662074696D65207A6F6E650012
:10056000D1D5131020205357495443482044454EB9
:1005700059202020D2D51610202020496E70757485
:100580002064656E7920202000D1D5041020204100
:1005900043434553532044454E59202020D2D5147F
:1005A0001020202020505245414C41524D20202007
:1005B0002000D1D50410202041434345535320440B
:1005C000454E59202020D2D5151020204C696D6948
:1005D00074202D2066756C6C202000C28E53890F0C
:1005E000438910758BD6758D97C28FD28E308FFD53
:1005F000C28E22C28E53890F438910758BEB758D85
:10060000CBC28FD28E308FFDC28E22C28E53890F05
:10061000438910E58AC4242BF58B758DEBC28FD2EC
:100620008E308FFDC28E22F9C3137004A250801841
:1006300014C0E0030303540F2482F8D0E0540704ED
:10064000F5F0E213D5F0FCE992E02275F00612070E
:100650000222C2A075F006120702D2A02212065290
:1006600012064B12065212064B12065212064B127B
:10067000065212064B12065275F01812070222C2D9
:10068000A075F04B120702D2A022755204123EDB75
:10069000C2A075F0C8120702D2A022755205123E00
:1006A000DB12067F75F01E12070212067F227552BA
:1006B00007123EDB12066922755206123EDB120655
:1006C0006F2212065D12065D22755207123EDB751F
:1006D0005206123EDB12066F12066F12066F2212CE
:1006E000066F12066322C2A1C26512065275F0128D
:1006F000120702D2A1C2652212065275F012120729
:1007000002221205DB201707C0F0122D99D0F0D578
:10071000F0F0227004A250B322C0E014120722D0DD
:10072000E022C0E0030303540F28F8D0E0C0E054F7
:100730000704F5F0E213D5F0FCD0E022E574B40034
:1007400003020831B40717C2AC12060B12060BD213
:10075000991208F4C25CD2B6126E9E02082EB40141
:1007600017C2AC12060B12060BD29912153AC25CD4
:10077000D2B6126E9E02082EB40317C2AC12060B3C
:1007800012060BD2991215BFC25CD2B6126E9E022F
:10079000082EB40217C2AC12060B12060BD2991225
:1007A000145BC25CD2B6126E9E02082EB40417C24D
:1007B000AC12060B12060BD29912149DC25CD2B673
:1007C000126E9E02082EB40517C2AC12060B12065A
:1007D0000BD29912085DC25CD2B6126E9E02082E30
:1007E000B40617C2AC12060B12060BD299121607EA
:1007F000C25CD2B6126E9E02082EB40817C2AC12AA
:10080000060B12060BD299126A9BC25CD2B6126E0C
:100810009E02082EB40917C2AC12060B12060BD2A8
:1008200099126A1FC25CD2B6126E9E02082E7574AF
:1008300000E56F6013B4010512330F8008B40205A0
:1008400012331E8000756F00122D9930470B20A8BF
:1008500008306205C26212334B12745F22C2B612B4
:10086000016275380074031253BCE51E1253BCE5D7
:100870001F1253BC74571253BC7881E623235403D0
:100880001253BC7882E630E402240A540F1253BC9F
:100890007881E6C4540375F00AA4F5F0E6540F25F8
:1008A000F01253BC7880E6C4540375F00AA4F5F046
:1008B000E6540F25F01253BC787FE6C4540775F058
:1008C0000AA4F5F0E6540F25F01253BC787EE6C476
:1008D000540775F00AA4F5F0E6540F25F01253BC46
:1008E0007882E603C454071253BCE5381253BC3077
:1008F00099FDD322126CDBC2B67538007403125313
:10090000BCE51E1253BCE51F1253BC74501253BCFD
:10091000747D1253BC900000E536600F9003E8141C
:1009200060099007D0146003900BB87E7D7F087536
:10093000F000C0F0126CD6B40203D38001C3D0E043
:1009400033F5F0A3DFEC1253BCDEE2E5381253BC02
:100950003099FD22C0F075F0DCD5F005B2B5126714
:10096000A4C0F0120B9ED0F030E7EED0F022AAF037
:10097000120954E5336530F5F0E534653145F06032
:100980000C120AC5853033853134120954120B63B9
:10099000120954120B8B120954120AD28AF022AA9D
:1009A000F0120954E5336530F5F0E534653145F072
:1009B000600C120AC5853033853134120954120B8C
:1009C0004F120954120B8B120954120AD28AF022C8
:1009D00079207530017531037532E09000DD120920
:1009E00054120AC5120954120B237900753001758F
:1009F00031047532009000FD120954120AC5120923
:100A000054120B2379E07530017531057532009071
:100A100001FD120954120AC5120954120B23853024
:100A20003385313422AAF0120954E5336530F5F0EC
:100A3000E534653145F0600C120AC58530338531E7
:100A400034120954120B0B8AF022AAF0120954E551
:100A5000336530F5F0E534653145F0600C120AC5B8
:100A6000853033853134120954120AF38AF022C0DA
:100A7000F075F00833C297928300D297D5F0F5D085
:100A8000F022C0F075F008C297D29700A28233D549
:100A9000F0F5D0F022D2B7D297D283D282D284227C
:100AA000E53133E5303322C3E5313322E53222121A
:100AB0000A6F120AA0120A6F120AA7120A6F120A0C
:100AC000AC120A6F22120A95C2847453120AAFD272
:100AD0008422120A95C2847458120AAFD284221258
:100AE0000A95C2847454120AAFE4120A6F120A8281
:100AF000D28422120A95C2847454120AAFE4120AF4
:100B00006F120A82F608D9F9D28422120A95C28499
:100B10007454120AAFE4120A6F120A82F208D9F969
:100B2000D28422120A95C2847454120AAFE4120AC3
:100B30006F120A82F0A3D9F9D28422120A95C0E07A
:100B4000C2847484120AAFD0E0120A6FD2842212D7
:100B50000A95C2847484120AAFE6120A6F08D9F9A2
:100B6000D28422120A95C2847484120AAFE2120A55
:100B70006F08D9F9D28422120A95C2847484120AA9
:100B8000AFE0120A6FA3D9F9D28422120A95C28467
:100B90007483120AAFD2841205DB1205DB22C284F1
:100BA0007457120A6F120A82D28422D283D282D25E
:100BB00097D2B7D284B2B575F0021205DBD5F0FA40
:100BC000C2B7B2B575F0021205DBD5F0FAD2B7B2F2
:100BD000B5227530017531DB753200120954120EE1
:100BE0006D7533FF7534FF22AE83AD8290DB007FDD
:100BF000207404F9747CF875300185833185823264
:100C0000120A4A787CE66E702508E66D702008E6C8
:100C1000601AB4FF028013167404F9747CF87530FE
:100C20000185833185823212099FC322D322A3A377
:100C3000A3A3DFBD80F490DB007F207404F9747CF3
:100C4000F8753001858331858232120A4A787CE654
:100C50006E700908E66D700408E6FC22A3A3A3A346
:100C6000DF0A7CFF2290DB007F207BFF7404F97495
:100C70007CF8753001858331858232120A4A787C8E
:100C8000E66E702C08E66D702708ECB4FF0D787CDA
:100C900076FF0876FF0876FF0874FFF67404F9748F
:100CA0007CF875300185833185823212099FC32219
:100CB000BBFF10787CE6B4FF0A08E6B4FF05C374F6
:100CC000209FFBA3A3A3A3DFA3BBFF02D322EB239D
:100CD0002354FC2400F5827583DB50020583787C65
:100CE000EEF608EDF608ECF608E4F67404F9747C08
:100CF000F875300185833185823212099FC32275D0
:100D0000830075F08E753002858331753200C0F036
:100D1000C083120954120E6DD0830583D0F0D5F034
:100D2000E475830075F0DA75300385833175320020
:100D3000C0F0C083120954120E6DD0830583D0F029
:100D4000D5F0E47533FF7534FF227583007582009A
:100D500075F08EC0F0C082C0837530028583317516
:100D60003200120954120AC5D083D082C082C083D7
:100D7000753000858231753200120954120B8BD008
:100D800083D08205830582D0F0D5F0C775830075C6
:100D9000820075F0DAC0F0C082C0837530038583AD
:100DA00031753200120954120AC5D083D082C08234
:100DB000C083753001858231753200120954120BDF
:100DC0008BD083D08205830582D0F0D5F0C77533F0
:100DD000FF7534FF2275830075820075F08EC0F0B8
:100DE000C082C0837530008583317532001209548A
:100DF000120AC5D083D082C082C08375300285823A
:100E000031753200120954120B8BD083D0820583C6
:100E10000582D0F0D5F0C775830075820075F0DAD1
:100E2000C0F0C082C08375300185833175320012F5
:100E30000954120AC5D083D082C082C083753003A2
:100E4000858231753200120954120B8BD083D08207
:100E500005830582D0F0D5F0C77533FF7534FF22C6
:100E6000120A95C2847450120AAFD28422120A95D3
:100E7000C2847481120AAFD28422120A95C2847489
:100E800084120AAFE8120A6FD9FAD28422AAF012A9
:100E90000954E5336530F5F0E534653145F0600C13
:100EA000120AC5853033853134120954120E7A1274
:100EB0000954120B8B8AF022120A95C284745412C0
:100EC0000AAFE4120A6FE4C0E0120A82D0F025F003
:100ED000D9F5D2842275830075820280067583005D
:100EE000758200E475F08D8582308583317532001E
:100EF000C082C083C0F0C0E0120954120AC51209B2
:100F0000547900120EB8D0F025F0D0F0D083D08202
:100F10000583D5F0D2858230858331753200C0E0FB
:100F2000120954120AC51209547920120EB8D0F0D1
:100F300025F07533FF7534FF2275830075820380B9
:100F400006758300758201E475F0DA858230858349
:100F500031753200C082C083C0F0C0E01209541263
:100F60000AC51209547900120EB8D0F025F0D0F05D
:100F7000D083D0820583D5F0D27533FF7534FF0559
:100F8000E02275830075F00075300085833175327D
:100F900000C0F0C083120954120E6DD0830583D0B7
:100FA000F0D5F0E47533FF7534FF75830075F0DA22
:100FB000753001858331753200C0F0C08312095449
:100FC000120E6DD0830583D0F0D5F0E47533FF7534
:100FD00034FF22120675754CFA3090FA75F005123E
:100FE00005DBD5F0FA754CFA2090FA222222222253
:100FF00022300A597881E6540FC0E0E6C4540375E4
:10100000F00AA4D0F025F0FD7882E630E402240A4C
:10101000540FFE901A007F3C7404F97400F8753088
:1010200001858331858232120A257800E26D7017BE
:1010300008E26E701208E2C42354E0F5F07882E60C
:10104000541F45F0F68006A3A3A3A3DFCB22120111
:1010500062120FF1120171FEAFF012690F7DFF0DE8
:10106000ED30E70122D27175F004A424DDF582E5AC
:10107000F03400F583C082C083787CE0F6A308E0FA
:10108000F6A308E0F6A308E0F6D083D082120FEEB4
:10109000787C8683088682787CB6FF0708B6FF03D3
:1010A000021107C3E58233F582E58333F583E582D8
:1010B00024E0F582E5833405F583787EE670480800
:1010C000E66044FB7402F9747CF875300185833165
:1010D000858232120A4A120FEFA3A3787CE60856E3
:1010E000B4FF03021107787C86F053F07F08E6C353
:1010F0009EC0E0E5F09FD0F0400445F07009787C98
:10110000E6A2E79271DBBD120FF0BD003DB2711295
:101110003286403320323020180E30330B204F05FA
:10112000307124800320711FA271924F92E0A2506F
:1011300092E1F5F013925065F030E00B205005126B
:10114000332D800312333C02105FED14C0E0030323
:1011500003540F2482F8D0E0540704FB7400D33307
:10116000DBFD307105FBE24B8004F4FBE25BF20235
:10117000105F120A6F120AA0120A6F120AA7D2E0B9
:10118000120A6F120AAC120A6F22120A95C28474F4
:1011900054121172E4120A6F120A82F608D9F9D2B7
:1011A0008422120A95C2847484121172E6120A6FA4
:1011B00008D9F9D2842290FC00753004753100758D
:1011C0003200C082C083754CFA120954120AC585D8
:1011D000306E85316D7908787C12095412118A12AB
:1011E00013B2D083D0827044C082C083788086835B
:1011F0000886821212634024787E868308868212D3
:1012000012634018121282E582600AE56BB56D0C1C
:10121000E56CB56E07D083D08202123E787EE6245C
:101220009AF61213F5126467D083D0820531E53146
:1012300070020530A3E5824583708712124575332D
:10124000FF7534FF22787E7600087600788076007D
:10125000087600087600087600756E04756D001239
:1012600013D122C082C083E5822400F582E5833455
:1012700080F5834005D083D08222D083D082900035
:101280000022E58275F008A4F582E5F0C58375F0CB
:1012900008A42583F583E5F03404F56CE582240089
:1012A000F582E5833400F5835002056C85836B225B
:1012B000126477D083D08222C082C08312138B70D5
:1012C000EF787E868308868212126340E3121282D0
:1012D00012166C787C76007880E518F608E519F629
:1012E0000876000876007408F9747CF8856C3085FF
:1012F000833185823212099F7404F97480F8856CF9
:1013000030858331858232120A4A75F004787C79FF
:1013100080E667600280990809D5F0F5121392788B
:101320007E8683088682A3121263787EA68308A62F
:101330008278808683088682121263787EE66583CF
:10134000700A08E665827004A31212637880A6838F
:1013500008A682C06EC06D856C6E856B6D1213D150
:10136000D0E0D0F0B56D09C5F0B56E028018C5F0BB
:10137000C06EC06D85F06EF56D787EE62499F6122C
:1013800013F5D06DD06ED083D08222121392121337
:10139000B222856E30856D31753200120954120A01
:1013A000C57908787C12095412118A853033853149
:1013B00034227881E61826182618261824556670D7
:1013C0000F7881E6186618661866186618649966BC
:1013D000221213D81213F5227881E618261826183F
:1013E00026182455F67881E6186618661866186679
:1013F000186499F622856E30856D317532001209B8
:1014000054120AC51209547908787C1211A21209E3
:1014100054120B8B120954120AD2853033853134A1
:101420002212138B7030787EE6C0E008E6C0E00838
:101430008683088682C3D0E09582F582D0E09583CA
:10144000F58350104582600CE5822400F582E58327
:101450003480F583C322900000D322C2B612142137
:10146000E433C0E075380074031253BCE51E125318
:10147000BCE51F1253BC74531253BCD0E01253BCD2
:1014800074001253BC74001253BCE5831253BCE5C4
:10149000821253BCE5381253BC3099FD22C2B6E526
:1014A000366004F4FF8004FF12124575380074039F
:1014B0001253BCE51E1253BCE51F1253BC745612E6
:1014C00053BCEF1253BCE5381253BC3099FD227463
:1014D00001C0E0787C75F008E4F608D5F0FBD0E0B8
:1014E000D32212142140E860E8788086830886823F
:1014F0001214F5C322C082C083E58275F008A4F5FA
:1015000082E5F0C58375F008A42583F583E5F03402
:1015100004F56CE5822400F582E5833400F5835000
:1015200002056C7408F9747CF8856C30858331850C
:101530008232120A4AD083D082221214217F0850AC
:10154000051212457F00787E865B08865C08865D02
:1015500008865EC2B675380074031253BCE51E12CD
:1015600053BCE51F1253BC74541253BCE5361253DE
:10157000BCEF1253BCE536603CE55E655CF5F0E51A
:101580005D655B45F0600B855E82855D831214F5B9
:1015900080031214D1855E82855D83A31212638558
:1015A000825E85835D787C75F008E61253BC08D5B1
:1015B000F0F8D536C4E5381253BC3099FDC322E5A6
:1015C000367007C2AF1214215005E536F4800C784E
:1015D00080A65D08A65E1213D1E536D2AFC0E0C288
:1015E000B675380074031253BCE51E1253BCE51FD8
:1015F0001253BC74551253BCD0E01253BCE53812E0
:1016000053BC3099FDD322C2B6753800740312530F
:10161000BCE51E1253BCE51F1253BC74581253BCD8
:101620007420232354FC041253BC74201253BC9026
:10163000DB007F207404F9747CF8753001858331F8
:10164000858232120A4A787CE61253BC08E61253AD
:10165000BC08E61253BC08E61253BC08A3A3A3A31C
:10166000DFD2E5381253BC3099FDD32212016278E3
:1016700082E630E402240A540FC4F97881E6C454A7
:101680000375F00AA4F5F0E6540F25F0C31349786A
:101690007DF67881E692E754C0F9787FE6C4540776
:1016A00075F00AA4F5F0E6540F25F049F97880E6C4
:1016B000C4540375F00AA4F5F0E6540F25F0F5F0D4
:1016C000787EE654702345F0787FF6787EE9F6223E
:1016D000C082C083E5301264B9E5311264B9787E06
:1016E000E61264B908E61264B908E61264B908E6BD
:1016F0001264B9120FD3D083D08222535A0F535998
:101700000F5318F053190FC2AFE5592324ADF8E574
:10171000184519F608A61A055953590FE559B55A2F
:1017200005055A535A0FD2AFC3E559955A500224B2
:101730001024F4500375640022E55AB5590574006D
:10174000780022C33324ADF8E6C0E008E6F8D0E024
:1017500022223051FDC2A075F006120702D2A075F8
:10176000F014120702E540C25122301703754BF006
:10177000122691205107740F30170580F31217526B
:1017800022C228A228B392A522D228A228B392A5C9
:1017900022B228A228B392A522F5F00303543FB445
:1017A000025BE53964086005E539B40D4DE5F08963
:1017B000F0C0F0300A1CC0E078D1E26013C33350AF
:1017C00005D0E00217E112062750F6D0E00217D24A
:1017D000D0E0D0F0A9F05403B4020D121781021822
:1017E000CCD0F0A9F00218CCB40106121789021867
:1017F000CCB403061217910218CC0218CAB40365C0
:10180000E53A64086005E53AB40DEFE5F089F0C00B
:10181000F0300A1CC0E078D2E26013C3335005D028
:10182000E002184312062750F6D0E0021830D0E04C
:10183000D0F0A9F05403B40211C229A229B392A690
:101840000218CCD0F0A9F00218CCB4010AD229A217
:1018500029B392A60218CCB40309B229A229B392E3
:10186000A680698065B40462E53B64086005E53BD9
:10187000B40D57E5F089F0C0F0300A1CC0E078D80C
:10188000E26013C3335005D0E00218AA12062750B5
:10189000F6D0E0021898D0E0D0F0A9F05403B402DA
:1018A0000FC22DA22DB392808022D0F0A9F0801C0F
:1018B000B40109D22DA22DB392808010B40309B2D5
:1018C0002DA22DB3928080048000D322C322797C84
:1018D000776BE4A25092E0A26A92E1A26B92E2A23C
:1018E0002792E3A24F92E4A26C92E5A26D92E709DF
:1018F000F709770009770009A73909A73A09A73B33
:101900000977007408F9747CF875300275318E75AA
:10191000320012099F7410F97482F8753002753123
:101920008E75320812096E22D24FD250C222C228BE
:10193000A228B392A5C223C229A229B392A6C22B80
:10194000C22DA22DB39280227408F9747CF87530F0
:101950000275318E753200120A4A787CB66BC978EE
:101960007DE6A2E09250A2E4924F78808639088604
:101970003A08863BE5397008A250B39228B392A585
:10198000E53A7008A250B39229B392A6E53B7008DD
:10199000A250B3922DB392807410F97482F875300E
:1019A0000275318E753208120A25787C76FF740133
:1019B000F9747CF875300275318E75320012099F0A
:1019C0002278CD75F010E4F208D5F0FB74FF78D5DD
:1019D000F278D6F222D24E6F20657874656E646517
:1019E000642020202020202020007565FF1219C1CE
:1019F000C20AC209120F4170611209D07401F97450
:101A000065F87530017531037532A0120A4A7410F9
:101A1000F974CDF87530017531037532A1120A25BC
:101A20007410F97492F87530017531037532C01273
:101A30000A257410F974A2F87530017531037532F6
:101A4000D0120A257402F97471F87530017531CE1F
:101A5000753200120A25D20AD2092222E8C0E078A3
:101A60006DE2F573D0E0F822E8C0E0786EE2F5733D
:101A7000D0E0F822E8C0E0786FE2F573D0E0F82219
:101A800075F00384B40104741A8017B4020474223C
:101A90008010B40304742A8009B4040474428002E0
:101AA000741A227403F9746AF875300075318C75F4
:101AB00032E5120A25786AE2121A80786DF2786BA4
:101AC000E2121A80786EF2786CE2121A80786FF265
:101AD000786AE224FD92017401F97469F8753000A6
:101AE00075318C7532E2120A257869E224FD92057F
:101AF000227403F9746AF875300075318C7532E51B
:101B000012096E7401F97469F875300075318C75BD
:101B100032E212096E22797C774809774E09777D87
:101B20000977A07404F9747CF875300075318D75EF
:101B3000322012099F7404F9747CF87530027531F3
:101B40008D75322012099F227404F9747CF8753067
:101B50000075318D753220120A4A797EE7647D2244
:101B6000E4A21D92E0A21E92E1A21F92E2797CF70C
:101B70007401F9747CF875300075318C7532E81297
:101B8000099F227401F9747CF875300075318C75E9
:101B900032E8120A4A797CE7A2E0921DA2E1921E85
:101BA000A2E2921F22797CE4A22E92E0A22F92E17F
:101BB000A23092E2A21592E392E492E5A23292E67A
:101BC000A23392E7F709E4A23192E0A23492E1A2B3
:101BD0003592E2A23692E3A23892E4A23892E5A2CC
:101BE0003992E6A23A92E7F709E4A23B92E0A23CDE
:101BF00092E1A23D92E2A23E92E3A23F92E4A24091
:101C000092E5A24192E7F709E4A24292E0A2029291
:101C1000E1A20392E2A24392E3A24592E4A2469299
:101C2000E5A24792E6A24492E7F77404F9747CF8BF
:101C300075300075318C7532EC12099F797CE4A205
:101C40004892E1A24992E2A24A92E3A24B92E4F4C2
:101C5000F709E4F4F709E4F4F77403F9747CF87510
:101C6000300075318C7532E912099F227404F974C1
:101C70007CF875300075318C7532EC120A4A797C2B
:101C8000E7A2E0922EA2E1922FA2E29230A2E3928A
:101C900015A2E69232A2E7923309E7A2E09231A2BE
:101CA000E19234A2E29235A2E39236A2E4A2E59256
:101CB00038A2E69239A2E7923A09E7A2E0923BA263
:101CC000E1923CA2E2923DA2E3923EA2E4923FA2C4
:101CD000E59240A2E6A2E7924109E7A2E09242A281
:101CE000E19202A2E29203A2E39243A2E49245A20D
:101CF000E59246A2E69247A2E792447403F9747C07
:101D0000F875300075318C7532E9120A4A797CE732
:101D1000F4A2E19248A2E29249A2E3924AA2E4929A
:101D20004B09E7F409E7F422797CF77401F9747C34
:101D3000F875300075318C7532E412099F227401F8
:101D4000F9747CF875300075318C7532E4120A4AEA
:101D5000797CE7227401F9745BF875300075318C79
:101D60007532FC12096E227401F9745BF87530004B
:101D700075318C7532FC120A2522785BE270067888
:101D80005CF208F222C2F0303F0475F03CA4AAF0E5
:101D900075F008A4FBACF0EA75F008A42CFAC37443
:101DA000FD9BFB74FF9A785CF2EB08F2227401F958
:101DB000745EF875300075318D75320012096E222F
:101DC0007401F9745EF875300075318D753200124A
:101DD0000A25227402F97478F875300075318C7513
:101DE00032FD120A257402F9747AF87530007531E3
:101DF0008D753201120A25227402F97478F8753053
:101E00000075318C7532FD12096E7402F9747AF81E
:101E100075300075318D75320112096E227401F929
:101E20007461F875300075318C7532F012096E747A
:101E300001F97462F875300075318C7532F412094D
:101E40006E7401F97463F875300075318C7532F673
:101E500012096E7401F97464F875300075318C756F
:101E600032F212096E227401F97461F8753000754E
:101E7000318C7532F0120A257401F97462F87530EC
:101E80000075318C7532F4120A257401F97463F807
:101E900075300075318C7532F6120A257401F974AB
:101EA00064F875300075318C7532F2120A2522748F
:101EB00001F97439F875300075318C7532F81209F2
:101EC0009F7401F9743AF875300075318C7532FAE7
:101ED00012099F7401F9743BF875300075318C75E7
:101EE00032FB12099F227401F97439F875300075BC
:101EF000318C7532F8120A4A7401F9743AF8753067
:101F00000075318C7532FA120A4A7401F9743BF883
:101F100075300075318C7532FB120A4A227402F951
:101F2000741EF875300075318C7532E012099F22ED
:101F30007402F9741EF875300075318C7532E01238
:101F40000A4A22C082C083E58275F008A42420F5E5
:101F500082500205F0A8F0E58375F008A42824005B
:101F6000F583787C76FF7401F9747CF87530008510
:101F7000833185823212099FA3A3A3A3A37401F91D
:101F8000747CF875300085833185823212099FD0C8
:101F900083D082C209220809E7C4F5F066540F70A5
:101FA0000D08E7F5F066540F7004DAEAE422E6540F
:101FB0000FC5F0540FC395F092087401227881790F
:101FC000277A03E6C4540FF309E6540FF30908DA3D
:101FD000F2792778A07A06E6540FF6E366700809CE
:101FE00008DAF4E4C25622792C78A57A06C3E3967F
:101FF0001918DAFA9208792C78A57A06E3540FB406
:102000000F08E6540FB40F108008E6540FB40F0BFE
:1020100080061819DAE680CB740122C3E396B4096E
:1020200002801214600FC3E3F5F0E695F0B40902E4
:1020300080031470E3E9B42704E4D256221918E3AC
:1020400066540F60F080D1121FBD701A30561720F1
:10205000311575185085831985821A1216FB754A39
:10206000B4D252D255E42204227408F9747CF87573
:10207000300075318C7532C0120A4A749EC3957255
:102080009572F8C374819572F9AA72121F9822741E
:1020900008F9747CF875300075318C7532C0120AFD
:1020A0004A122047227405F9747CF87530007531A6
:1020B0008C7532C012099F227403F97481F875304F
:1020C0000075318C7532C512099F22C082C083E52C
:1020D000822420F582E583347DF5837401F9743C14
:1020E000F8753000858331858232120A4AD083D058
:1020F00082C082C083E58275F008A42420F5825056
:102100000205F0A8F0E58375F008A4282400F58303
:102110007408F9747CF87530008583318582321239
:102120000A4AD083D082124F4622C082C083E58201
:1021300075F008A42420F582500205F0A8F0E5838C
:1021400075F008A4282400F5837408F97494F875D0
:102150003000858331858232120A4AD083D08222B0
:10216000C082C083E58275F008A42420F582500265
:1021700005F0A8F0E58375F008A4282400F5837421
:1021800006F9747CF8753000858331858232120A35
:102190004AD083D082227405F9747CF875300075BA
:1021A0003100753220120A4A749EC395729572F8F6
:1021B000C374819572F9AA72121F9822751B20753B
:1021C0001C009000007405F9747CF8753000851CC3
:1021D00031851B32120A4A749EC395729572F8C3F8
:1021E00074819572F9AA72121F986018E51B240871
:1021F000F51B5002051CA3E583B40FC9E582B4A00A
:10220000C47401221220CBE42220090280AE751B87
:1022100000751C0075699F756A0FE569251BC2E092
:10222000F582E56A351CF583C082C083E58224000F
:10223000F582E583341BF5837402F9747CF87530FC
:1022400001858331858232120A4A787C868308862A
:10225000821220CB749EC395729572F8C3748195D7
:1022600072F9AA72121F987005D0F0D0F022D083B4
:10227000D082C3E58313F583E58213F58220081429
:10228000E58245836023E58224FFF569E58334FF19
:10229000F56A8007A385821B85831CC3E569951BAE
:1022A000E56A951C400302221A740122300A247840
:1022B0009479B275F00AE3B4FF028017B43C0F08BA
:1022C00009D5F0F2900FE878DBE2F53CE4226654A1
:1022D0000F60EC740122751B25751C0090000074C2
:1022E00003F97481F8753000851C31851B32120AA0
:1022F0004A1220476018E51B2408F51B5002051CF4
:10230000A3E583B40FD9E582B4A0D47401221220CE
:10231000CBE42278A0E6540FB40F030223AD2009CA
:102320000280B3751B00751C0075699F756A0FE507
:1023300069251BC2E0F582E56A351CF583C082C0C1
:1023400083E5822400F582E583343BF5837402F94A
:10235000747CF8753001858331858232120A4A789F
:102360007C86830886821220CB1220477005D0F02D
:10237000D0F022D083D082C3E58313F583E58213A6
:10238000F582200814E58245836022E58224FFF56A
:1023900069E58334FFF56A8007A385821B85831C6A
:1023A000C3E569951BE56A951C4002808274012291
:1023B00078947A0579A8E6540FC4F5F008E6540F2E
:1023C00045F0F70809DAEF22C2A3C263C2A2C266CF
:1023D000C2A1C265D2B775F0021205DBD5F0FA20B2
:1023E000B72BD217D2A3C263C2A2D266D2A1C26552
:1023F000D2A4C264120675B2B575F00F1205DBD512
:10240000F0FA30B7EF12249EC2AF027054D2A0127D
:102410000EDD700C12244D121B4870041219EA22B2
:10242000C217754CFA75F0641205DBD5F0FAC2A03C
:10243000C2A2C26675F0641205DBD5F0FAD2A0D252
:10244000A2C266D2B71205F320B7D58095121B83BE
:10245000121C6C121D3EA2E0924CA2E1924DA2E22F
:10246000924E121D67121DC0121E66121EE6121D2C
:10247000D37410F974B2F87530017531CE7532200D
:10248000120A25121F30121AA3121D7A22C2A3C2E9
:1024900063C2A2C266C2A1C265D2A4C26422D2171C
:1024A00012638940E8C2A3C263C2A2C266C2A1C2CB
:1024B00065D2A4C264C01EC01F787C9000007A0858
:1024C000E6F008A3DAFA12258C787C9000007A08EE
:1024D000E0F608A3DAFA9000001260CE1220A512EE
:1024E00020B8D01FD01E121F1D12614B12124512B0
:1024F0000BD222751E30751F30C21DC21EC21FC2F4
:102500002EC22FC230C215C232C233C231D234C23F
:1025100035C236C238C239C23AC23BC23CC23DC2E1
:102520003EC23FC240C241C242C243C244C245C28F
:1025300046C247C248C249C24AC24B78787422F2A6
:10254000087400F2787A7406F2087400F2C24CC281
:102550004DC24E785B7404F2785E7409F27861744F
:1025600001F278627402F278637404F2786474049D
:10257000F2753907753A00753B0074017869F27895
:102580006AF2E408F208F2C20AC20922120F8212A9
:1025900024F3121F1D121B60121BA5C2E0A24C9255
:1025A000E0A24D92E1A24E92E2121D28121D541299
:1025B0001DAD121E1D121EAF121DF8121AF1121BB4
:1025C00016126B5422306804C268800975F00C2022
:1025D000B205D5F0FAD322C322E8C0E0E9C0E0EAB0
:1025E000C0E02005372001341225C5502575520062
:1025F000786AE2600C75F0031205DBD5F0FA123B45
:10260000E57869E2600C75F0031205DBD5F0FA128B
:102610003D5AD0E0FAD0E0F9D0E0F8223075F3C0AE
:1026200082C083E5717008127246400312263B1285
:102630001A5C12721AD083D08280D730040C300515
:1026400009D270C26F78690226533001F4D26FC28A
:1026500070786AE2B40F028013B41007125135D2B9
:102660005E802D75F00384E5F0B40007125218D295
:102670005E801DB401071250B4D25D8013B4021005
:1026800012503F400B7859E583F208E582F2D25FA1
:1026900022D2608008C260122703753D00C216D2A4
:1026A00068754CFA7440301702740CF549C25EC26A
:1026B00051E54960391225D9205E3375F0031205C2
:1026C000DBD5F0FA12073C2017032016183051E131
:1026D00020601B754960121752B40B0D75F008127B
:1026E00005DBD5F0FAD25E80051226F680C3C25D06
:1026F000D2AF754CFA22533D07F8E53D24A0C8F649
:10270000053D2278A075F00874FFF608D5F0FB228D
:10271000305D09201C03D21C22C25D22C21C22D2C1
:10272000608004D268C260C216754CFAD21B744035
:10273000301702740CF549122703753D00C25EC2C2
:102740005DC251C25FC26112073C20170320162DE3
:102750001225D9205E29205D26205F2330512A785A
:1027600069E27004C251802120601475496012171B
:1027700052B40B1275F0081205DBD5F0FAD25E7573
:102780004CFA12690F221226F6E54960F212690F1F
:102790003061FD80B0C0F088F0C0F0C2AF75770046
:1027A000785CE2F54DF5F008E2F54ED2AF45F0D099
:1027B000F0A8F0D0F07009B227202706C20B8002E3
:1027C000D227202704D2A78003757703D268D2626C
:1027D000223016012278A0760A087603800778A0B6
:1027E000760A0876010875F06484F608E5F075F05D
:1027F0000A84F608A6F0753D05D216227518C07534
:102800001900751A011216FB22754800C25475187A
:10281000C0751900751A021216FB22D252754AB4FD
:1028200075185075190F751AFF1216FB22C20C127B
:102830002795203D0C75181075190F751AFF121683
:10284000FB22203D0C75182075190F751AFF121602
:10285000FB2275186075190F751AFF1216FB227589
:10286000187075190F751AFF1216FB22126B54752A
:1028700018C0751900751A0E1216FB22787CF20822
:10288000F2123F9D7518C0751900751A501216FB8B
:1028900030450022401A306916C269206A11C2AF61
:1028A000754D00754E01D2AFC227757700D2A722B1
:1028B0002069FCC20C122795D26922122A66400DAB
:1028C000122CC24008122F35400312319622122AD0
:1028D00071400D122CCD4008122F4040031231A13F
:1028E00022301708C37865E4F2022A7FA290301DD7
:1028F00001B37865E233F2B4FF03022903022A7FB1
:10290000022B3C2020032024F7D224300A1CC0E0F4
:1029100078CDE26013C3335005D0E0022B3C1206A1
:102920002750F6D0E002292AD0E07861E260D1B4E5
:10293000012DD20D1227FC30271C203B11C2AF7590
:102940004D00754E08D2AFC227757700D2A7785ECA
:10295000E2F548022B3C20390312281B022B3CB421
:10296000021A1228BB400F302F03205009206B069B
:1029700012282D022B2E122842022B3CB40308C22F
:1029800050122852022B3CB40706757A0175700369
:10299000B4090C205003203A03022A58022B3CB4FD
:1029A0000A02743DB40E09D3122894740E022A58F8
:1029B000B4340874001227D1022B3CB435087410CB
:1029C0001227D1022B3CB4360874111227D1022BE6
:1029D0003CB4370874201227D1022B3CB4381B7446
:1029E00001F9747CF875300075318C7532F1120A7A
:1029F0004A787CE61227D1022B3CB4391B7401F9CA
:102A0000747CF875300075318C7532F1120A4A7891
:102A10007CE61227DE022B3CB43C0612286C022B0B
:102A20002EB43D13205008D25012285F022B2EC224
:102A300050122852022B2EB43E0D304507E41228C6
:102A40007C022B2E022B3CB43F0E30450874FF1243
:102A5000287C022B2E022B3C751890751909F51A4B
:102A60001216FB022B3C7861E2B40B03A22422C3B2
:102A7000222050097861E2B40D03A22422C32270FF
:102A8000E22020033024DCC224300A1CC0E078CDD0
:102A9000E26013C3335005D0E0022B3C12062750EE
:102AA000F6D0E0022AA8D0E07861E26024B4010800
:102AB000C20D122809022B3CB40203022B3CB403C2
:102AC00007D25012285F8074B40908205052303A5F
:102AD0004F8069B40A02743DB40E09C3122894747D
:102AE0000E022B20B432028053B43302804EB43431
:102AF000028049B435028044B43602803FB43702C4
:102B0000803AB438028035B439028030B43C028057
:102B10002BB43D028026B43E028021B43F02801CCB
:102B20007518A0751909F51A1216FB022B3C100630
:102B300003022B3C12696A1206AED2062230170835
:102B4000C37866E4F2022CDBA291301E01B37866F2
:102B5000E233F2B4FF03022B5F022CDB022D98203C
:102B600020032025F7D225300A1CC0E078CEE26091
:102B700013C3335005D0E0022D9812062750F6D02B
:102B8000E0022B86D0E07862E260D1B4012DD20D54
:102B90001227FC30271C203B11C2AF754D00754E2B
:102BA00008D2AFC227757700D2A7785EE2F5480257
:102BB0002D9820390312281B022D98B4021A1228CE
:102BC000BB400F302F03205009206B0612282D0226
:102BD0002D8A122842022D98B40308C2501228529E
:102BE000022D98B40706757A01757003B4090C209C
:102BF0005003203A03022CB4022D98B40A02743D0B
:102C0000B40E09D3122894740E022CB4B434087490
:102C1000001227D1022D98B4350874101227D10262
:102C20002D98B4360874111227D1022D98B43708A4
:102C300074201227D1022D98B4381B7401F9747CCA
:102C4000F875300075318C7532F5120A4A787CE6D9
:102C50001227D1022D98B4391B7401F9747CF875D0
:102C6000300075318C7532F5120A4A787CE61227ED
:102C7000DE022D98B43C0612286C022D8AB43D1356
:102C8000205008D25012285F022D8AC250122852BA
:102C9000022D8AB43E0D304507E412287C022D8AAD
:102CA000022D98B43F0E30450874FF12287C022D87
:102CB0008A022D9875189075190AF51A1216FB02DA
:102CC0002D987862E2B40B03A22522C3222050097A
:102CD0007862E2B40D03A22522C32270E220200311
:102CE0003025DCC225300A1CC0E078CEE26013C378
:102CF000335005D0E0022D9812062750F6D0E0029E
:102D00002D04D0E07862E26024B40108C20D1228DC
:102D100009022D98B40203022D98B40307D2501271
:102D2000285F8074B40908205052303A4F8069B44B
:102D30000A02743DB40E09C3122894740E022D7C4D
:102D4000B432028053B43302804EB434028049B4AA
:102D500035028044B43602803FB43702803AB4383A
:102D6000028035B439028030B43C02802BB43D027D
:102D70008026B43E028021B43F02801C7518A075E5
:102D8000190AF51A1216FB022D98100603022D9847
:102D900012696A1206AED2062230470E204803128C
:102DA00028E1204903122B3D80061228E1122B3D19
:102DB000301708C37867E4F2022F4EA292301F0149
:102DC000B37867E233F2B4FF03022DD2022F4E0232
:102DD000300B2020032026F7D226300A1CC0E078D2
:102DE000CFE26013C3335005D0E002300B12062748
:102DF00050F6D0E0022DF9D0E07863E260D1B40162
:102E00002DD20D1227FC30271C203B11C2AF754D6F
:102E100000754E08D2AFC227757700D2A7785EE260
:102E2000F54802300B20390312281B02300BB40284
:102E30001A1228BB400F302F03205009206B0612B6
:102E4000282D022FFD12284202300BB40308C25075
:102E500012285202300BB40706757A01757003B45C
:102E6000090C205003203A03022F2702300BB40A2A
:102E700002743DB40E09D3122894740E022F27B4A5
:102E8000340874001227D102300BB43508741012C4
:102E900027D102300BB4360874111227D102300B3F
:102EA000B4370874201227D102300BB4381B7401D8
:102EB000F9747CF875300075318C7532F7120A4A56
:102EC000787CE61227D102300BB4391B7401F974F7
:102ED0007CF875300075318C7532F7120A4A787CAF
:102EE000E61227DE02300BB43C0612286C022FFDDE
:102EF000B43D13205008D25012285F022FFDC2505B
:102F0000122852022FFDB43E0D304507E412287CF2
:102F1000022FFD02300BB43F0E30450874FF12281B
:102F20007C022FFD02300B75189075190CF51A12E2
:102F300016FB02300B7863E2B40B03A22622C322F5
:102F40002050097863E2B40D03A22622C32270E266
:102F50002020033026DCC226300A1CC0E078CFE2F5
:102F60006013C3335005D0E002300B12062750F631
:102F7000D0E0022F77D0E07863E26024B40108C289
:102F80000D12280902300BB4020302300BB4030700
:102F9000D25012285F8074B40908205052303A4F42
:102FA0008069B40A02743DB40E09C3122894740EE9
:102FB000022FEFB432028053B43302804EB4340295
:102FC0008049B435028044B43602803FB437028071
:102FD0003AB438028035B439028030B43C02802BD8
:102FE000B43D028026B43E028021B43F02801C75AD
:102FF00018A075190CF51A1216FB02300B100603F7
:1030000002300B12696A1206AED206301708C37876
:1030100068E4F20231AFA285302A01B37868E23366
:10302000F2B4FF0302302D0231AF023271202003CF
:10303000202CF7D22C300A1CC0E078D7E26013C3F2
:10304000335005D0E002327112062750F6D0E0026C
:103050003054D0E07864E260D1B4012DD20D122753
:10306000FC30271C203B11C2AF754D00754E08D2B5
:10307000AFC227757700D2A7785EE2F548023271B9
:1030800020390312281B023271B4021A1228BB40E5
:103090000F302F03205009206B0612282D023263B7
:1030A000122842023271B40308C25012285202326E
:1030B00071B40706757A01757003B4090C205003CA
:1030C000203A03023188023271B40A02743DB40C12
:1030D00003023271B40E09D3122894740E0231889F
:1030E000B4340874001227D1023271B43508741058
:1030F0001227D1023271B4360874111227D102326C
:1031000071B4370874201227D1023271B4381B749D
:1031100001F9747CF875300075318C7532F3120A40
:103120004A787CE61227D1023271B4391B7401F956
:10313000747CF875300075318C7532F3120A4A7858
:103140007CE61227DE023271B43C0612286C023291
:1031500063B43D13205008D25012285F023263C27C
:1031600050122852023263B43E0D304507E4122853
:103170007C023263023271B43F0E30450874FF1294
:10318000287C02326302327175189075190DF51A98
:103190001216FB0232717864E2B40B03A22C22C334
:1031A000222050097864E2B40D03A22C22C32270BD
:1031B000E2202003302CDCC22C300A1CC0E078D77F
:1031C000E26013C3335005D0E0023271120627507B
:1031D000F6D0E00231D8D0E07864E26024B401088F
:1031E000C20D122809023271B40203023271B40313
:1031F00007D25012285F8079B40908205057303A1E
:1032000054806EB40A02743DB40C028064B40E099A
:10321000C3122894740E023255B432028053B43370
:1032200002804EB434028049B435028044B4360280
:10323000803FB43702803AB438028035B439028016
:1032400030B43C02802BB43D028026B43E02802183
:10325000B43F02801C7518A075190DF51A1216FBE3
:1032600002327110060302327112696A1206AED27E
:1032700006C22020570122C25775184075190075E3
:103280001A001216FB22E8C0E07861E264036018BD
:103290007862E2640360117863E26403600A786430
:1032A000E264036003C38001D3D0E0F8221206F881
:1032B000300A0C12653B400390FFF112658022C07A
:1032C000531232DDD05322300A1312653B40039073
:1032D000FFF11265805005F5531265D722E5537052
:1032E000057553108023B41005755311801BB4115C
:1032F000057553208013B420057553FF800BB4FF70
:103300000575530080037553FF126640E55322C2D2
:103310005075186075190F751AFA1216FB22D250E3
:1033200075187075190F751AFA1216FB22C25075AE
:10333000186075190F751AE01216FB22D250751815
:103340007075190F751AE01216FB22E4A22792E09D
:10335000A22892E1A22992E2A22D92E3F575757658
:1033600005123F13740350041240922212406C78ED
:103370008DE6C0E0304812D0E0C0E054071233A31D
:10338000D0E0C0E054071233A3304914D0E0C0E0CD
:10339000C454071235F1D0E0C0E0C454071235F12F
:1033A000D0E022A224301D01B34007D320E10A025D
:1033B00035F0C320E2030235F0301D01B3301708A9
:1033C000C37865E4F202353340060235350235F044
:1033D0002020032024F7D224300A1CC0E078CDE25C
:1033E0006013C3335005D0E00235F012062750F6C3
:1033F000D0E00233F7D0E07861E260D1B4012DD2A1
:103400000D1227FC30271C203B11C2AF754D0075F3
:103410004E08D2AFC227757700D2A7785EE2F54892
:103420000235F020390312281B0235F0B4021A12BB
:1034300028BB400F302F03205009206B0612282D87
:103440000235E21228420235F0B40308C2501228B5
:10345000520235F0B40706757A01757003B4090C91
:10346000205003203A030235250235F0B40A0274D5
:103470003DB40E09D3122894740E023525B43408D5
:1034800074001227D10235F0B4350874101227D118
:103490000235F0B4360874111227D10235F0B43772
:1034A0000874201227D10235F0B4381B7401F97466
:1034B0007CF875300075318C7532F1120A4A787CCF
:1034C000E61227D10235F0B4391B7401F9747CF887
:1034D00075300075318C7532F1120A4A787CE6122B
:1034E00027DE0235F0B43C0612286C0235E2B43D0A
:1034F00013205008D25012285F0235E2C250122821
:10350000520235E2B43E0D304507E412287C023504
:10351000E20235F0B43F0E30450874FF12287C02F9
:1035200035E20235F0751890751909F51A1216FB77
:103530000235F070FB2020033024F5C224300A1C31
:10354000C0E078CDE26013C3335005D0E00235F01F
:1035500012062750F6D0E002355CD0E07861E260D8
:1035600024B40108C20D1228090235F0B402030286
:1035700035F0B40307D25012285F8074B4090820D4
:103580005052303A4F8069B40A02743DB40E09C3F8
:10359000122894740E0235D4B432028053B433022C
:1035A000804EB434028049B435028044B43602807F
:1035B0003FB43702803AB438028035B439028030E3
:1035C000B43C02802BB43D028026B43E028021B47C
:1035D0003F02801C7518A0751909F51A1216FB0216
:1035E00035F01006030235F012696A1206AED206F3
:1035F00022A225301E01B34007D320E10A02383E43
:10360000C320E20302383E301E01B3301708C378EE
:1036100066E4F2023781400602378302383E2020FA
:10362000032025F7D225300A1CC0E078CEE26013D3
:10363000C3335005D0E002383E12062750F6D0E0E2
:10364000023645D0E07862E260D1B4012DD20D128D
:1036500027FC30271C203B11C2AF754D00754E086A
:10366000D2AFC227757700D2A7785EE2F54802385C
:103670003E20390312281B02383EB4021A1228BB1E
:10368000400F302F03205009206B0612282D0238DE
:103690003012284202383EB40308C25012285202A7
:1036A000383EB40706757A01757003B4090C2050D2
:1036B00003203A0302377302383EB40A02743DB461
:1036C0000E09D3122894740E023773B434087400B0
:1036D0001227D102383EB4350874101227D10238AF
:1036E0003EB4360874111227D102383EB43708743C
:1036F000201227D102383EB4381B7401F9747CF8CB
:1037000075300075318C7532F5120A4A787CE612F4
:1037100027D102383EB4391B7401F9747CF8753036
:103720000075318C7532F5120A4A787CE61227DE74
:1037300002383EB43C0612286C023830B43D1320E7
:103740005008D25012285F023830C250122852025C
:103750003830B43E0D304507E412287C0238300280
:10376000383EB43F0E30450874FF12287C023830D2
:1037700002383E75189075190AF51A1216FB0238B0
:103780003E70FB2020033025F5C225300A1CC0E026
:1037900078CEE26013C3335005D0E002383E120603
:1037A0002750F6D0E00237AAD0E07862E26024B475
:1037B0000108C20D12280902383EB4020302383E45
:1037C000B40307D25012285F8074B4090820505205
:1037D000303A4F8069B40A02743DB40E09C312280E
:1037E00094740E023822B432028053B43302804EF5
:1037F000B434028049B435028044B43602803FB408
:103800003702803AB438028035B439028030B43C93
:1038100002802BB43D028026B43E028021B43F02D8
:10382000801C7518A075190AF51A1216FB02383E8D
:1038300010060302383E12696A1206AED206221240
:103840003957123A0A123ABD22123964123A171243
:103850003ACA22B20E300A1CC0E078D1E26013C32B
:10386000335005D0E00238D212062750F6D0E002DD
:103870003874D0E0E53970030238E024F84005E5FB
:10388000390238EBE539B40904A20B8056B40A04B6
:10389000A20D804FB40C03D38049B40D0B3022032A
:1038A000023971D222D3803BB40E04A20C8034B40E
:1038B0000F08C3E57A6001D38029B4100AE5784582
:1038C00079C36001D3801CB41105125370801402B7
:1038D0003971B40D06202203023971C222C380035C
:1038E000A250B39228B392A5023971300E66304BC4
:1038F000033050175351037851A2E282524030A254
:10390000E082534012A2E182544018C228A228B398
:1039100092A57600023971B60102801D76017550BC
:10392000408016B60202801176027550A0800AB659
:103930000302800576037550F0D262E55023F550FE
:1039400020E00AC228A228B392A5023971D228A287
:1039500028B392A5023971E539B40B07D228A22801
:10396000B392A522E539B40B07C228A228B392A5C9
:1039700022300A1CC0E078D2E26013C3335005D075
:10398000E00239EE12062750F6D0E0023990D0E07E
:10399000E53A70030239FC24F84005E53A023A079B
:1039A000E53AB40904A20B8056B40A04A20D804F74
:1039B000B40C03D38049B40D0B302303023A24D254
:1039C00023D3803BB40E04A20C8034B40F08C3E5AB
:1039D0007A6001D38029B4100AE5784579C3600183
:1039E000D3801CB411051253708014023A24B40D14
:1039F00006202303023A24C223C38003A250B392B9
:103A000029B392A6023A24023A24E53AB40B07D22B
:103A100029A229B392A622E53AB40B07C229A2290A
:103A2000B392A622300A1CC0E078D8E26013C333F8
:103A30005005D0E0023AA112062750F6D0E0023A33
:103A400043D0E0E53B7003023AAF24F84005E53B84
:103A5000023ABAE53BB40904A20B8056B40A04A2A8
:103A60000D804FB40C03D38049B40D0B302B0302EF
:103A70003AD7D22BD3803BB40E04A20C8034B40FBF
:103A800008C3E57A6001D38029B4100AE578457946
:103A9000C36001D3801CB411051253708014023A24
:103AA000D7B40D06202B03023AD7C22BC38003A242
:103AB00050B3922DB39280023AD7023AD7E53BB485
:103AC0000B07D22DA22DB3928022E53BB40B07C287
:103AD0002DA22DB392802222B40207205E07C25D80
:103AE000C25F023B66C082C08390EA60E53D6063CE
:103AF00024FB405F78A0E6540F758300F582D53D26
:103B000002805075F00AA4F58275830008E6540F10
:103B10002582F582D53D02803AE58275F00AA4F54A
:103B20008285F08308E62582F58250020583D53D23
:103B3000028020E58275F00AA4F582C0F0E5837565
:103B4000F00AA4D0F025F0F58308E62582F582502E
:103B50000205837859E583F208E582F2C25EC25D10
:103B6000D25FD083D08222C289C28BD293C2B422C8
:103B7000C0F075F0FAD5F0FD75F064D5F0FDD0F029
:103B800022123B70123B70123B70123B70123B7062
:103B9000123B7022D293C2B475F0051205F320B225
:103BA000061205F330B203D5F0F11205F322C0F08E
:103BB00075F008A2E7B392B4C293123B70C2B4D2BC
:103BC00093123B70C0E0E430B201040030B2010453
:103BD0000030B20104D36003D5E001C3D0E033D597
:103BE000F0D1D0F022D293C2B4D2B2123B70C293C1
:103BF000123B81D293123B8120170330701C788CCA
:103C00007601087480F608A2A3B392E4F6749008D3
:103C1000F608F608F608F6023C5A788C7603087621
:103C200080087480A26392E5A2A3B392E4201708EF
:103C3000A26692E1A22792E0F60874802017122073
:103C4000700FE55254074480A26592E5A2A1B39299
:103C5000E4F6087480F608F608F675F007788C7EAE
:103C6000007F00E62EFEE6123BAEF62FFF08D5F0F1
:103C7000F2EED333123BAEF8EFD33368707B788C1F
:103C8000B6FF760562E56224FE50147562022019C3
:103C90000ED2197518C0751900751A031216FB207B
:103CA0001708786AE26003307003023D567892E6A6
:103CB00020E36D20E25D20E13E788DE6B600380815
:103CC000B64220757A017570037518B075190075C4
:103CD0001A001216FB7518C0751900751A0712160E
:103CE000FB8073B6551108B6000D087959E6F30844
:103CF00009E6F3D25FD26F805DE5626014D5621190
:103D000030190EC2197518C0751900751A041216EB
:103D1000FB8043788D863D08D25E79A07A04800BC3
:103D2000788DD25D75720579947A05D26F75F00F32
:103D3000E6C4540FF755F0F5F009E6540FF755F0C7
:103D4000F5F00908DAEAE5F0B40F051977EEC25D7F
:103D5000786AE2123AD8123B9422D293C2B4D2B219
:103D6000123B70C293123B81D293123B8120171FEA
:103D7000306F23788C7611087480F608A2A3B39272
:103D8000E4F6749008F608F608F608F6023DDF78C7
:103D90008C7615023D9A788C7613087680087480AC
:103DA000A26392E5A2A3B392E4206F14A26492E10D
:103DB000A2A4B392E0201708A26692E1A22792E0A3
:103DC000F6087480206F0FE55254074480A2659274
:103DD000E5A2A1B392E4F6087480F608F608F67539
:103DE000F007788C7E007F00E62EFEE6123BAEF6F2
:103DF0002FFF08D5F0F2EED333123BAEF8EFD333FA
:103E000068706C788CB6FF670561E56124FE50141C
:103E1000756102201A0ED21A7518C0751900751A2C
:103E2000051216FB7869E26003306F03023ED77813
:103E300092E620E36C20E25C20E14F788DE6B6004C
:103E40002C08B64214757A017570037518C075197F
:103E500000751A071216FB807EB6551108B6000DC4
:103E6000087959E6F30809E6F3D25FD2708068E575
:103E7000616014D56111301A0EC21A7518C0751917
:103E800000751A061216FB023ED7D270788D864056
:103E9000D2518043788D863D08D25E79A07A048025
:103EA0000B788DD25D75720579947A05D27075F0B4
:103EB0000FE6C4540FF755F0F5F009E6540FF75527
:103EC000F0F5F00908DAEAE5F0B40F051977EEC26B
:103ED0005D7869E2123AD8123B9422786AE224FDB6
:103EE0004020E2600C75F0031205DBD5F0FA123BBE
:103EF000E57869E2600C75F0031205DBD5F0FA1283
:103F00003D5A22306F0C7518B0751900751A0012E1
:103F100016FB22D293C2B4D2B2123B70C293123BB0
:103F200081D293123B81788CE576540FC44407F616
:103F300008E57523A2E392E5A2E292E3542AD2E7D0
:103F4000F608E575A2E392E1A2E492E3542AD2E7EF
:103F5000F608E575A2E692E1A2E792E3540AD2E7F9
:103F6000F6748008F608F608F675F007788C7E007F
:103F70007F00E62EFEE6123BAEF62FFF08D5F0F2EC
:103F8000EED333123BAEF8EFD33368700B788CB6B8
:103F9000FF06123B94C38004123B94D3227576082B
:103FA000787CE2F575123F137400400512406C8076
:103FB00003124092757609787DE2F575123F13740D
:103FC00001400512406C8003124092227576047500
:103FD00075FF123F13740250041240922212406C7B
:103FE000788F7954E6F30809E6F3087956E6F30882
:103FF00009E6F3788DE6A2E092E25414F5F008E6C3
:1040000023A2E592E0540345F0F5F07858E265F01C
:10401000C0E0E5F0F2D0E030E21FC0E0C0F0E5F033
:1040200075F04930E20375F04A7518C075190085BE
:10403000F01A1216FBD0F0D0E05403700302406B6C
:10404000E5F05403B4030575F0488013B402057518
:10405000F047800BB4000575F04B800375F04C758C
:1040600018C075190085F01A1216FB22F5F0244AC3
:10407000F8E2B40205227402F22250FA7402F2E568
:10408000F02432F5F07518C075190085F01A121673
:10409000FB22F5F0244AF8E26017D5E013F2E5F0D0
:1040A000243CF5F07518C075190085F01A1216FB3E
:1040B000F222D293C2B4D2B2123B70C293123B81AD
:1040C000D293123B81788CE576540FC44403F608F2
:1040D0007680087480A26392E5A2A3B392E4A266FC
:1040E00092E1A22792E0F6087480A26592E5A2A16F
:1040F000B392E4F6087480F608F608F675F00778CF
:104100008C7E007F00E62EFEE6123BAEF62FFF0807
:10411000D5F0F2EED333123BAEF8EFD333687071C3
:10412000788CB6FF6C7892E620E33020E22020E124
:1041300060788DE6B6005A08B6551108B6005208E8
:104140007959E6F30809E6F3D25F804A8043788D17
:10415000863D08D25E79A07A04800B788DD25D7599
:10416000720579947A0575F00FE6C4540FF755F08F
:10417000F5F009E6540FF755F0F5F00908DAEAE52D
:10418000F0B40F051977EEC25D7870E2123AD8806C
:1041900005123B94D322123B94C322700575641E12
:1041A0008002D21222C298C299322017F830991890
:1041B000C299205C05753500800EC0E0C0D075D076
:1041C000101244ACD0D0D0E020980132C298205CCC
:1041D000FAC0D0C0E0E8C0E0305B05C25B754200C9
:1041E000E54624FE4003754602E54220E712E5421B
:1041F0005407232492C0E074003443C0E0E59922C0
:10420000543F23232485C0E074003442C0E0E59984
:10421000221563024384024384D563FAB5450975C8
:104220007B0175420002438A0243A2B462FA024350
:1042300084024384B42AF1024384F56324C6E5630F
:1042400040E624F5E56350E005630243847820F2FC
:1042500015630243847821F215630243847822F2C5
:1042600015630243847823F215630243847824F2B1
:1042700015630243847825F215630243847826F29D
:1042800015630243840243B80002422B000242310C
:10429000000242340002423A00024211000242117E
:1042A00000024211000242110002424D000242553A
:1042B0000002425D000242650002426D000242754A
:1042C0000002427D00024219000242190002421916
:1042D000000242190002421900024219000242196A
:1042E000000242190002421900024219000242195A
:1042F000000242190002421900024219000242194A
:104300000002421900024219000242190002421939
:104310000002421900024219000242190002421929
:104320000002421900024219000242190002421919
:104330000002421900024219000242190002421909
:1043400000024219000242190002421900024219F9
:1043500000024219000242190002421900024219E9
:1043600000024219000242190002421900024219D9
:1043700000024219000242190002421900024219C9
:10438000000243B805422545F545D0E0F8D0E0D01D
:10439000D032800E802A802D803080328034804060
:1043A000803EB4090875450075420080D7B44208C4
:1043B00075450075428080CC75450075420080CA05
:1043C000B51EDF80BFB51FDA80BAF54380B6F5446D
:1043D00080B2B545CD7546201243E275420080AAF1
:1043E00080D6854337126EC3D25CE537B4460302EC
:1043F000543CB44704126ED922B4500E8544361290
:104400006E9EC2ACC25C75740722B45312854436EA
:10441000E544700A126E9EC2ACC25C75740222B48E
:10442000540E854436126E9EC2ACC25C7574012275
:10443000B4550E854436126E9EC2ACC25C757403D0
:1044400022B4560E854436126E9EC2ACC25C7574A0
:104450000422B4570E854436126E9EC2ACC25C75FF
:10446000740522B4580E854436126E9EC2ACC25CEE
:1044700075740622B44E21854436E544B4000B120F
:104480006E9EC2ACC25C75740822B4010B126E9EA3
:10449000C2ACC25C7574092224BF24E64004854482
:1044A0003622C25C22C5382538C53822E53524F0CD
:1044B000400EE5352324CBC0E074003444C0E02234
:1044C000759906C25C753500D2B622802F80348083
:1044D0003680388039803E804680488051804F80C9
:1044E0004D804B80468050800E024573753503F534
:1044F000991244A5053522740002452175380074CF
:104500000380ECE51E80E8E51F80E40245D7E5382E
:1045100075350F80DA12173912419B883680D0E545
:104520003680C9E536A25092E080C1753503A836C1
:104530000536E676FF80B8E536C313603214700B9B
:10454000A22492E0B392E1440480D614700BA22519
:1045500092E0B392E1440880C8147008A22692E069
:10456000440C80BD147008A22C92E0440C80B274FC
:10457000FC80AEE5361470257408306912306A0488
:104580004406809D306B044403809644078092A2C9
:104590006A92E0A26B92E1A22792E28084147015E5
:1045A0007410A22492E0A22592E1A22692E2A22C0B
:1045B00092E302452114700D7418A21992E0A21A18
:1045C00092E102452114700BA26C92E0A26D92E27E
:1045D000024521E4024521E537B441067535040260
:1045E00044EFB4422AE536600330121B53590F538F
:1045F0005A0FC2AFE55AB55906D2AFD302460705E6
:104600005A535A0FD2AFC375641E74420244ECB4BD
:104610004455200AF7E536C3137022B3926712326D
:1046200086404020323D30330B204F0530673480C8
:104630000320672FA2679250924F0246639267143D
:10464000C0E0030303540F2482F8D0E0540704FAB7
:104650007400D333DAFD306705FAE24A8004F4FAD5
:10466000E25AF6E53780A5B44B0280030246F5E531
:104670003654F8B40812E5365407602B146047141A
:10468000604B1460670244C0B420030244C0B428E5
:1046900013E536A2E09250756F015003756F02E585
:1046A000370244EC0244C0751AF4C26BC26A206936
:1046B0006BC2AF754D00754E01D2AFC22775770042
:1046C000D2A7D2688056751AF3D26B80DF751AF2C2
:1046D000D26AC26B206945C2AF754D00754E01D2DA
:1046E000AFC227757700D2A7D2688030751AF1D291
:1046F0006AC26B801FB4430FB53603754703753527
:10470000077536A80244EFB44A23E536701C206BC7
:1047100019751AF0C20C20690312279575181075C7
:10472000190F1216FBE5370244EC0244C0B44506EB
:104730007535060244EFB4510675350C0244EFB4EA
:104740004D0EE536121799E5375002B2E702460CD6
:10475000B44C0675350E0244EFB4460280C9B44726
:104760000280C4B44F08C252C253C25480B902443A
:10477000C0E566C2736002D273E553F554C255209A
:104780005F0C205D1B305E030247FD024D95120653
:10479000E67859E2F58308E2F5821220CB0249302F
:1047A0001206E61223B012220960081222AC703001
:1047B000024930206F05206C0A8003206D05124EDF
:1047C00009501AC082C0831206B8122695D083D031
:1047D00082305E0CE53D60081220477003024930CC
:1047E000754B3CD5471475183075190085471A125A
:1047F00016FB754703D253754AB4024D801206E684
:10480000E53D60F6B402061262A7024D95206F19CD
:10481000201603303413B4051078A0B60A0B08B67E
:1048200001028008B6030280030248C808E675F05A
:104830000AA4082675F00AA40826C5F0703B78A1E2
:10484000B60339201609C0F0124DC4D0F0502A85A5
:10485000F05385F0541206AE20160F7518C0751966
:104860000385531A1216FB024D957518C07519026F
:1048700085531A1216FB024D95024D78201609C079
:10488000F0124DB0D0F050F185F05320160E75188F
:10489000C075190685531A1216FB800C7518C07561
:1048A000190585531A1216FB1265DB124DF6D2A2BA
:1048B000C266C2A1D2651206B8122723A25D725E3B
:1048C000500302477F024D951223137047206F0556
:1048D000206C0A8003206D05124E0950531206B851
:1048E000C082C083122723D083D082305D23C08250
:1048F000C0831206E61223B0D083D082749EC39583
:10490000729572F8C374819572F9AA72121F986039
:104910001F0247E07869207002786AE2B40F0A1239
:1049200050F1C25ED25D0247A3B4100280F180E173
:10493000306F33300A1CC0E078D9E26013C33350C3
:1049400005D0E002496612062750F6D0E00249522F
:10495000D0E0757602786BE27870F2121A68125223
:104960006650030247E0307033300A1CC0E078DA4A
:10497000E26013C3335005D0E002499C1206275071
:10498000F6D0E0024988D0E0757603786CE2787062
:10499000F2121A7412526650030247E012708440F9
:1049A00003123B67E53C0470030247E0754B00755A
:1049B0004703C254C253205502C252C082C0831260
:1049C0004EB0D083D0825006124D31024D95C08238
:1049D000C083120BE8D083D0825006124D31024DB5
:1049E00095E58224CEE58334FF5017124DF740122F
:1049F000C213C2141232865006124D22024D950285
:104A00004C3C1228BB5012124D22024BD3124D1CAB
:104A1000024BD3124D16024BD3206BF1302F0320E3
:104A200050F1306F037860E2307002E53C6009239A
:104A30001206274003024A41024A88124D10024BD7
:104A4000D3300AF73015F43040F112538E4039A2BA
:104A50006F304101B35031300A1BC0E078D6E260BC
:104A600012C3335004D0E080D212062750F7D0E0B2
:104A7000024A75D0E0C082C083126D2FD083D082ED
:104A80005006124D27024BD330157212538E406DD3
:104A9000126CDBA2E09213A2E19214A26F304101EA
:104AA000B3C0E09207501E1253705019303C0EE410
:104AB000A21392E0A21492E1B402028008D0E012A4
:104AC0004CFE024BD3D0E0B40005200722802BB46B
:104AD000012220071A7518C0751900751A091216D7
:104AE000FB203C06124D2C024BD3124DA6800E1219
:104AF0006C208009B402ED2007DB126C7B300A7E4B
:104B000012538E4079300A1CC0E078D5E26013C39E
:104B1000335005D0E0024B7E12062750F6D0E0025B
:104B20004B24D0E0207316A26F9272858367858232
:104B300068124DA21206C9756602024D957566008F
:104B4000E5836567F5F0E582656845F07006124D0E
:104B500036024BD37518C0751900751A0C1216FB66
:104B600030720C7518B0751900751A001216FB1208
:104B70004D5B75181085671985681A1216FB305041
:104B80000EC2A3C263C2A2C266D2A4C264800CD207
:104B9000A3C263C2A2C266C2A4C264A26F920CD2B4
:104BA0000B124D9E12279530470620A80312334B57
:104BB000123F03124D5B75181085831985821A12F6
:104BC00016FB1206AE30450BC082C083124FD1D007
:104BD00083D082124E005009124F4630E103024D3D
:104BE0009512328640F8C2A1D265D2A4C264755231
:104BF00000123EDB1220CBC082C083122723D08359
:104C0000D082205F09205D17205E2C024D95120690
:104C1000E67859E2B5831D08E2B58218024C3C746F
:104C20009EC395729572F8C374819572F9AA721237
:104C30001F986008024D8012204770F8301524E458
:104C4000A21392E0A21492E1B40305126CAA80139D
:104C5000B40205126C20800BB40105126C7B80033A
:104C6000126BF4300A1CC0E078D3E26013C33350F7
:104C700005D0E0024D8012062750F6D0E0024C82AB
:104C8000D0E0304225E5824583601F306F037860B5
:104C9000E2307002E53C6009231206274003024C13
:104CA000A4024CAA124D04024D951228CE500F12A8
:104CB0004D0A75F01E12070212069B024D95B25066
:104CC000123F0330501A75187085831985821A12A5
:104CD00016FBC2A3C263D2A1C265D2A4C26480186B
:104CE00075186085831985821A1216FBD2A3C263D8
:104CF000D2A1C265C2A4C2641206AE024D95126969
:104D000005024D39126905024D39126905024D3906
:104D1000126905024D39126905024D391269050201
:104D20004D391269058012126905800D12690580DE
:104D30000812690580031269057566007567FF75BD
:104D400068FF12383F123F0375182085831985824A
:104D50001A1216FB12069B12384922204A03206FB2
:104D600016E553046011146565600C7518C075195B
:104D70000185531A1216FB2212690512068A801544
:104D800012690512383F12068A1238497566007595
:104D900067FF7568FFC25EC25DE554F55322126974
:104DA00005221269052212690575F03212070222E6
:104DB0007408F9747CF875300175310375329812F6
:104DC0000A4A80127408F9747CF875300175310351
:104DD000753290120A4A7881E60856085604601423
:104DE0001206B8122695305E09E53D60051220478F
:104DF0006002C322D32222E582249CE58334FF2271
:104E0000E582249CE58334FF22A24DE58245836040
:104E100010E582249CE58334FF5004A24C8002A25A
:104E20004E22E5822582F582E5833583F583E5828E
:104E30002582F582E5833583F583E5822400F582BA
:104E4000E583345BF5837404F97400F875300185EB
:104E50008331858232120A25227881E654C0F58397
:104E60007882E630E402240A2323543C4583F58308
:104E70007881E6C4540375F00AA4F5F0E6540F25D2
:104E8000F0030303F5F053F0E085F082540345830B
:104E9000F5837880E6C4540375F00AA4F5F0E6546F
:104EA0000F25F04582F58222C39582E5F095832295
:104EB00012538E5003024F38124E227800E2B4FF94
:104EC00003024F38120162124E59787CA68308A65D
:104ED000827800E2F58308E2F58208E2F5F008E264
:104EE000124EA8502B7800E2F58308E2F582787C18
:104EF00086F008E6124EA850417802E2F58308E2F7
:104F0000F582787C86F008E6124EA8402D024F38D4
:104F10007800E2F58308E2F582787C86F008E612F4
:104F20004EA840167802E2F58308E2F582787C8686
:104F3000F008E6124EA85002C322D322785F74FF15
:104F4000F208F2F5F022300AF3C082C083C3E58292
:104F500033F582E58333F583E5822400F582E5832A
:104F6000349AF5837402F9745FF8753001858331E2
:104F7000858232120A25D083D082E5822418E58307
:104F800034FC4005785F74FFF27860E2F5F018E2D7
:104F900022E5822418E58334FC74FFF5F05031C01B
:104FA00082C083C3E58233F582E58333F583E582EE
:104FB0002400F582E583349AF5837402F9745FF86E
:104FC00075300185833185823212096ED083D0829B
:104FD00022E5822400F582E58334BAF5837401F971
:104FE000747CF8753001858331858232120A4A78E3
:104FF0007CE660422323C0E05403F5F0D0E054FC8B
:105000002400F582E5F034CAF5837404F9747CF861
:10501000753001858331858232120A4A787CE60830
:1050200086F0787CF208E5F0F275F0021205DBD527
:10503000F0FA123F9D2274FF787CF208F280EAE5D4
:1050400073B4220575F0048013B42A0575F0068048
:105050000BB4420575F00C800375F0027836E2540B
:105060000F704F08D5F0F7E2540F75F00AA4F582DF
:1050700075830008E2540F2582F582E58275F00AF7
:10508000A4F58285F08308E22582F582500205832B
:10509000E58275F00AA4F582C0F0E58375F00AA4F4
:1050A000D0F025F0F58308E22582F58250020583D1
:1050B000C322D3227836E573B4220A757204799636
:1050C00075F0088024B42A0A757205799475F00A7F
:1050D0008017B4420C757205799475F00A783C809B
:1050E00008757203799875F006E2F70809D5F0F9AA
:1050F00022789479C275F00AE3F60809D5F0F979B7
:10510000CCE3F57222789479C275F00AE6F30809C7
:10511000D5F0F9E57279CCF3221250B4749EC395A0
:10512000729572F8C374819572F9AA72121F98224F
:10513000D083D082221250B4125105122703C082AC
:10514000C083753D017836E2540F70E408E2540FD5
:1051500070DE08E2540FC4F5F008E2540F45F0F594
:105160008308E2540FC4F5F008E2540F45F0F582CD
:10517000C27978A07900C3E5829410F582E5839422
:1051800027F58340030980EEE5822410F582E5834C
:105190003427F583E96004D279F6087900C3E58203
:1051A00094E8F582E5839403F58340030980EEE5F6
:1051B0008224E8F582E5833403F583E920790460ED
:1051C00004D279F6087900C3E5829464F582E58318
:1051D0009400F58340030980EEE5822464F582E5BE
:1051E000833400F583E92079046004D279F608E578
:1051F0008275F00A842079026002F608E5F0F6E88C
:105200002461F53DD083D0822279A077000975F022
:105210000577FF09D5F0FA221250B4125105125247
:105220000975F008E573B4220478368013B42A04B3
:105230007838800CB44204783E8005783675F006E4
:10524000753D06E2540F700608D5F0F7800979A085
:10525000E2F70809D5F0F92212521812204722125B
:105260005135122047227870E2700302532624FD44
:105270004048C082C0831206B812532AD083D0821D
:10528000205F26205E1B305D41749EC3957295722F
:10529000F8C374819572F9AA72121F98702C025388
:1052A0002612204770240253267859E2B5831B0842
:1052B000E2B5821665827012806CC082C0831206CD
:1052C000B81272E8D083D08250030253287870E27B
:1052D000B40F0C125258604E125119604980EBB451
:1052E000100712525F603F80E175F00384E5F0B46F
:1052F000000712525870D3802DB401071251197053
:10530000C98023B4021EC082C08312503FE582854B
:1053100083F0D083D08240B2658270AEE5F06583C1
:1053200070A8800280A4C322D322754932D268308B
:105330006109C261C07612073CD076E549D3601896
:10534000C25FC25EC25D1225C550E41240B2205F4A
:1053500006205E03305DD8C3C0D0A8767405B802BD
:10536000027404D0D0400512406C80031240922297
:10537000E579457860167871E2F5F008E245F0606D
:105380000BD37872E2957918E2957822C322E582F0
:10539000B4E807E583B40F02D322C322C538253809
:1053A000C53822E54B24E94008D2A3C263D2A2C289
:1053B000663098EFC298E59912539C223099FDC24D
:1053C00099F59912539C22C2A3C263C2A2C266C2BB
:1053D000B675380074051253BCE51E1253BCE51FA8
:1053E0001253BC2212060B12060B12060B1253C7E5
:1053F000E5371253BCE5381253BC3099FD22120F29
:1054000041025407120EDDC0E01253C7E5371253B4
:10541000BCD0E01253BCE5381253BC3099FD2212C7
:10542000060B1253C7E5371253BC797CE71253BC05
:1054300009DDF9E5381253BC3099FD22751A007563
:105440004B19D217E539600B54F87007C228A2280F
:10545000B392A5E53A600B54F87007C229A229B3AC
:1054600092A6D2A0C28EC28CC2ADC2ABC2ACC2AF39
:105470007581CD90547EC082C08375D00032D2AF8A
:10548000D28C126E9EC2ACD2991253E4B2B5754B57
:1054900019D2980254BBB40922F5381253A3B51E91
:1054A000271253A3B51F211253A3B4461B1253A3B3
:1054B000AF381253A36F70101253E4D2B6D2A3C206
:1054C00063D2A2C2661253A3B40ACBF5381253A317
:1054D000B51EF51253A3B51FEF1253A3F537B46DE4
:1054E0000302556BB46E03025584B46F030255BBBF
:1054F000B47003025608B4710302561CB47303025D
:10550000562DB4740302562FB47503025643B47675
:105510000302565BB4770302566FB47803025683D6
:10552000B479030256A4B47A030256C0B46C0302E1
:1055300056D4B46B030256F6B46A03025731B46909
:105540000302574DB468030257ACB467030257C453
:10555000B466030257DFB465030258A3B4640302C0
:10556000601BB461030260760254BBAF381253A3D0
:105570006F70F51253E4D2B675F01E1205DBD5F04C
:10558000FA0270541253A3FD1424E0402B1253A3CB
:105590002400FC7B001253A3FEAF381253A36F709C
:1055A000178EF0EDF9747CF88B308C3185F0321267
:1055B0000A4A12541F754B190254BB1253A3FD140F
:1055C00054E070F41253A32400FC247140EA7B02DF
:1055D0001253A3FEEDFA787C1253A3F608DAF9AF62
:1055E000381253A36F70D1C2A3C263C2A2C2668E27
:1055F000F0EDF9747CF88B308C3185F03212099F14
:105600001253ED754B1980B0AF381253A36F70A8C9
:10561000120CFF1253E4754B190254BBAF381253EE
:10562000A36F7009125404754B190254BB80891280
:1056300053A3FD1424E040481253A32400FC7B0133
:105640000255951253A3FD1454E070341253A32451
:1056500000FC2425402A7B030255D0AF381253A307
:105660006F701D0256801253ED754B190254BBAF7B
:10567000381253A36F70091253FE754B190254BBB5
:105680000255B879207D071253A3F309DDFCAF382A
:105690001253A36F70EA1264BA40E5120143125329
:1056A000ED0254BBAF381253A36F70D412016212D3
:1056B000060B1253C7E5371253BC1208790254BBCC
:1056C000AF381253A36F70661212451253E4754B34
:1056D000190254BB1253A3FE1253A3FD1253A3FC91
:1056E000AF381253A36F7046120C6540411253E459
:1056F000754B190254BB1253A3FE1253A3FDAF38CE
:105700001253A36F7028120C3612060B12060B12DE
:1057100053C7E5371253BCEE1253BCED1253BCEC29
:105720001253BCE5381253BC3099FD0254BB0255EC
:10573000B8AF381253A36F70F512060B12060B1296
:1057400053C7E5371253BC1216200254BBAF3812B0
:1057500053A36F70D9120ED560027401C0E0120F0E
:105760003960027402D0F045F0700A120D4A121B23
:1057700016121245E4C0E01253C7E5371253BCD0ED
:10578000E0C0E01253BCE5381253BC75F0031205BB
:10579000DBD5F0FA1253C7E5371253BCD0E01253F1
:1057A000BCE5381253BC3099FD0254BB1253A3FD23
:1057B0001454E070271253A32400FC2471401D7B75
:1057C000000255D01253A3FD1454E0700F1253A3DE
:1057D0002400FC242540057B010255D00255B8AFBA
:1057E000381253A36F70F512060B12060B1253C733
:1057F000E5371253BC74011253BC744E1253BC747F
:105800007D1253BC74481253BC74321253BC7400E2
:105810001253BC748D1253BC74201253BC74DA1230
:1058200053BC74001253BC740F1253BC74A01253B7
:10583000BC74801253BC74001253BC74001253BC6D
:1058400074201253BC74001253BC74001253BC7405
:10585000001253BC74001253BC74001253BC740089
:105860001253BC74001253BC74001253BC74001267
:1058700053BC74001253BC74001253BC7400125316
:10588000BC74001253BC74001253BC74001253BC9D
:1058900074001253BCE5381253BC3099FD0254BB5E
:1058A0000255B81253A3F5831253A3F5822460E581
:1058B0008334F040EB125B8C1253A3FD1454E07060
:1058C000DF78001253A3F208DDF9AF381253A36F4B
:1058D00070CE1253E475F0051205DBD5F0FA1253C1
:1058E000ED751A01300AB93009B6125C00125BE698
:1058F000125B9A1220CB789479007A0A75F00FE344
:10590000540FF652F00809DAF643F0F0E5F00478A7
:1059100094797C7A05121F98600B1259BB5006755A
:105920001A040258A0125BE6125B9A1220CB78A0F0
:10593000790A7A0675F00FE3540FF652F00809DA87
:10594000F643F0F0E5F00478A079817A03121F980D
:10595000600B125A595006751A060258A0125BE6DF
:10596000125C49751A650254BBC0E07830E583F2D9
:1059700008E582F2D0E022C0E07832E583F208E563
:1059800082F2D0E022C0E07830E2F58308E2F582CE
:10599000D0E022C0E07832E2F58308E2F582D0E080
:1059A00022E5822400F582E583341BF58322E5821B
:1059B0002400F582E583343BF58322125B9AAB83A6
:1059C000AC82901B00C083790075300385833175EC
:1059D0003200900061120954120AC5120954120BC8
:1059E000239000617A80E0A3F5F0E0A36C7005E5F8
:1059F000F06B6017DAF0D0830583740024C0E58370
:105A000034C550C17405125B08D322D083EA2AF54D
:105A1000F0E4C395F0F582125969789479007A0A16
:105A200075F00FE3540FF652F00809DAF643F0F080
:105A3000E5F004600C12220E700A7406125B08D3A3
:105A40002212220EE5822582F582E5833583F583D5
:105A50001259A1125977025E20125B9AAB83AC8275
:105A6000903B00C083790075300385833175320027
:105A7000900061120954120AC5120954120B2390A6
:105A800000617A80E0A3F5F0E0A36C7005E5F06BAF
:105A90006017DAF0D0830583740024C0E58334A551
:105AA00050C17405125B08D322D083EA2AF5F0E4D2
:105AB000C395F0F58212596978A0790A7A0675F0D3
:105AC0000FE3540FF652F00809DAF643F0F0E5F070
:105AD00004601D122323701BAB83AC82125B9AEB14
:105AE000B58306ECB58202C3227404125B08D3228C
:105AF000122323E5822582F582E5833583F583121F
:105B000059AE125977025E20F51A22C082C083E591
:105B1000831264B9D083D082C082C083E5821264CC
:105B2000B9D083D08222C082C0837F00E58224F076
:105B3000C0E0E58334D8C0E05007D083D0820F8026
:105B4000EBD0E0D0E07F00E5822418C0E0E58334AC
:105B5000FCC0E05007D083D0820F80EBD0E0D0E0D3
:105B60007F00E582249CC0E0E58334FFC0E050075D
:105B7000D083D0820F80EBD0E0D0E0E58275F00AD0
:105B800084C0F0F5F0D0F0D083D08222C0E0783429
:105B9000E583F208E582F2D0E022C0E07834E2F555
:105BA0008308E2F582D0E0227881E61264B9788237
:105BB000E61264B97883E61264B978A0E61264B993
:105BC00078A1E61264B978A2E61264B978A3E61265
:105BD00064B978A4E61264B978A5E61264B9120F24
:105BE000D322120FD32274001253BC74001253BC80
:105BF00074001253BC74001253BC74001253BC22C4
:105C000075831B75821B75F040C0F0C082C0837520
:105C10003001858331753200120954120AC5D083D0
:105C2000D082C082C0837530038582317532001204
:105C30000954120B8BD083D08205830582D0F0D516
:105C4000F0C77533FF7534FF227401F97418F875C5
:105C50003000753100753200120A4A7401F9741966
:105C6000F87530017531D97532FF120A4AAC181235
:105C70005B9AE5822420F582E583347DF583C0823A
:105C8000C0837401F9743CF87530008583318582D6
:105C900032120A4AD083D0827401F97410F8753038
:105CA0000085833185823212096E7810E2F5F0E5C5
:105CB00018253CC395F0F518125B9AE58275F0083B
:105CC000A42420F582500205F0A8F0E58375F008C1
:105CD000A4282400F5837408F9747CF875300085D5
:105CE0008331858232120A4A787CE5187A082608C0
:105CF000DAFCF518789479007A0A75F00FE3540FFE
:105D0000F652F00809DAF643F0F0E5F00412640503
:105D100078A0790A7A0675F00FE3540FF652F0086E
:105D200009DAF643F0F0E5F00412640D7408F97432
:105D30007CF875300085833185823212099F787C2A
:105D4000E5187A08C39608DAFBF518125B9AC3E5E2
:105D50008233F582E58333F583C3E58233F582E54B
:105D60008333F583E5822400F582E583245BF583A4
:105D7000C082C0837404F9747CF875300185833166
:105D8000858232120A4AD083D0827404F97412F8E0
:105D900075300185833185823212096E787C7912E3
:105DA000E5197A0426F5F0E3C5F0C395F00809DAA1
:105DB000F3F5197401F97418F87530007531007530
:105DC000320012099F7401F97419F87530017531A8
:105DD000D97532FF12099F75831B75821B75F040C0
:105DE000C0F0C082C08375300385833175320012E4
:105DF0000954120AC5D083D082C082C08375300195
:105E0000858231753200120954120B8BD083D082F7
:105E100005830582D0F0D5F0C77533FF7534FF22B6
:105E2000125993E5828583F0125985C39582C0E0AB
:105E3000E5F09583D0F045F07002C3225003025F75
:105E40003B125993C0E0C3E58224FEF582E583341A
:105E5000FFF583D0E0125977E5828583F0125985EA
:105E6000B58207E5F0B58302C322125985AF8312CC
:105E70005993EFB58310AE82900034787CE0F6A39E
:105E800008E0F6025E9E7EFE8F8305837402F9743D
:105E90007CF8753003858331753200120A4A790027
:105EA0007530038F31753200900061120954120A67
:105EB000C5120954120B238F837582001259857DF8
:105EC00000E5836F7002AD82ED2461F58275830079
:105ED00050020583C3EE9D20E05A03FCC082C083BC
:105EE000A3A3E0FAA3E0FBD083D082EAF0A3EBF017
:105EF000A3DCE9EE2461F582758300500205837806
:105F00007CE6F0A308E6F079007530038F31753236
:105F100000900061120954120B77120954120B8B76
:105F2000853033853134125993EFB5830302600F06
:105F30000F025E6F7408125B08D322125985AF837B
:105F4000125993EFB58310AE82900034787CE0F65E
:105F5000A308E0F6025F6F7E008F8315837402F959
:105F6000747CF87530038583317532FE120A4A79E4
:105F7000007530038F3175320090006112095412A0
:105F80000AC5120954120B231259857DFEE5836F51
:105F90007002AD82ED2461F58275830050020583A5
:105FA000C3ED9E20E06B03FCC0E0C3E58224FEF558
:105FB00082E58334FFF583D0E0C082C083E0FAA39A
:105FC000E0FBA3EAF0A3EBF0D083D082DCDAEE248E
:105FD00061F58275830050020583787CE6F0A308A2
:105FE000E6F079007530038F317532009000611250
:105FF0000954120B77120954120B8B8530338531FB
:1060000034125993EFB5830302600F1F025F40C340
:10601000227409125B08D3220255B81253A3F583E8
:106020001253A3F582AF381253A36F70EBC01EC09A
:106030001F85831E85821F121F1D7401F9747CF851
:10604000753000753100753200120A4A787CE6C35B
:10605000951EC3951FD01FD01E251E251FF6740147
:10606000F9747CF875300075310075320012099FA3
:106070001253E40254BB1253A3F583AF381253A357
:106080006F709512060B12060B12060B1253C7E522
:10609000371253BC74001253BCE51A1253BC74007F
:1060A0001253BC74001253BC74001253BC7400121F
:1060B00053BCE5381253BC3099FD0254BB9060C507
:1060C000C082C083327581CD75D000027054C08209
:1060D000C083E5822420F582E583347DF583740155
:1060E000F9743CF875300085833185823212099F3E
:1060F000D083D082C082C083E58275F008A42420BA
:10610000F582500205F0A8F0E58375F008A4282474
:1061100000F5837404F9747CF8753000858331854B
:10612000823212099FA3A3A3A3747C2404F5F07404
:1061300004F9E5F0F8753000858331858232120963
:106140009FD083D082C209124F9122120EDDC0E08F
:106150007401F9747CF875300075310075320012E5
:106160000A4A787CE6D0F0C395F0F67401F9747CA5
:10617000F875300075310075320012099F22300A1F
:106180001CC0E078D3E26013C3335005D0E0026254
:106190002C12062750F6D0E002619DD0E0124DF699
:1061A000D2A3C263C2A1D265D2A4C2641206B8123D
:1061B0002723205D06205E3502622C1206F812228B
:1061C000097069124E004064206F05206C0A80033C
:1061D000206D05124E0950561206B8122695305EF3
:1061E0004BE53D6047122047704202622EE53D605C
:1061F0003B1206F81223137033124E00402E206F0C
:1062000005206C0A8003206D05124E0950201206ED
:10621000B8122723305D15749EC395729572F8C32A
:1062200074819572F9AA72121F986002D3223042CB
:1062300039E58245836033306F037860E230700265
:10624000E53C600923120627400302625002626A9D
:1062500012383F123F0375182085831985821A1260
:1062600016FB12069B12384980C2B250C3123F037C
:1062700030501A75187085831985821A1216FBC260
:10628000A3C263D2A1C265D2A4C26480187518608B
:1062900085831985821A1216FBD2A3C263D2A1C2CA
:1062A00065C2A4C264C32278A0E6B40A1708E6B4A3
:1062B0000545123286400912617E40041206AE2264
:1062C00012068A2275F00AA4F5F008E625F0B463F8
:1062D00026D2A3C263C2A2D266C2A1D265D2A4C290
:1062E00064C0E01206B81227239000001220CB20D1
:1062F0005D09205E35D0E012068A221206F8749EEF
:10630000C395729572F8C374819572F9AA72121FBF
:106310009870E2304D441206B8122695305ED612BF
:1063200006F812204770CE02635A1206F8E53D6067
:10633000C412204770BF304D211206B812272330F7
:106340005DB31206F8749EC395729572F8C374819A
:106350009572F9AA72121F98709B1206B8D0E012BB
:10636000068A2212614B7518C0751900751A0A1237
:1063700016FB1206AE22753C007860E4F2787C755C
:10638000F00876FF08D5F0FA22751E30751F30C26E
:106390006FC27075F005C0F0D2A3C263C2A2D2660C
:1063A000D2A1C265D2A4C264126376122723D0F0B0
:1063B000205D09205E06D5F0DD02640012642540F0
:1063C0003F1206AE7881E6B4FF05C32275F005C022
:1063D000F0122723D0F0205E06D5F0F3026400E52A
:1063E0003DB4021C78A0E624F6401508E624F640E9
:1063F0000F78A0E62430F51E08E62430F51FC322EE
:1064000012068AD3227894797C7A05800678A0795E
:10641000817A03E608540FC4F5F0E608540F45F0FE
:10642000F709DAEF22205D31305E3AE53D6006245F
:10643000FD24FC403012640D1206B875F005C0F062
:1064400012271FD0F0205D11205106D5F0F0026414
:1064500065121752B40B0E8003126405753C007868
:1064600060E4F2C322D32212647775F0641205DB74
:10647000D5F0FA12065D2275F03C120702C2A07533
:10648000F03C120702D2A075F014120702C2A075E8
:10649000F03C120702D2A075F014120702C2A075D8
:1064A000F014120702D2A075F014120702C2A075F0
:1064B000F014120702D2A02222227825E254C070E2
:1064C00078E275F00A84C445F0787EF67824E254C8
:1064D000C07066E275F00A84C445F0787FF67823D0
:1064E000E254E07054E275F00A84C445F07880F616
:1064F0007822E2604454E07040E275F00A84C445BA
:10650000F0C0E07820E2030354C0D0F045F0788179
:10651000F67821E2602354F0701FE275F00A84C41B
:1065200045F0C0E07826E254F8700EE2C42354E04F
:10653000D0F045F07882F6C322D32290000075F0A7
:1065400019C0F07402F9747CF875300185833185C7
:106550008232120A4A787DB6FF02800E18E5533067
:106560000A05B4FF02E565666011E5822410F58234
:1065700050020583D0F0D5F0C8C322D0F0A3D322B7
:10658000300A4DE58224FFF582E58334FFF58375FB
:10659000F019E5822480E58334FE500590000080E8
:1065A0000AE5822410F58250020583C0F07402F9D6
:1065B000747CF8753001858331858232120A4A78FD
:1065C0007DB6FF02800518E6B55307D0F0D5F0C2BE
:1065D000C322D0F0A3D32222026608E57B60F975BE
:1065E0007B001264BA40F112014302660B7822E28A
:1065F0001264B87821E21264B87823E21264B878A1
:1066000024E21264B802662F1201627881E6C45453
:1066100003E6540F7882E6C45401E6540F7880E60E
:10662000C4540FE6540F787FE6C4540FE6540F307D
:106630000A0A12653B50051265D780031266402294
:10664000E553B4FF0690040702667FB4000690028B
:106650008702667FB4100690029002667FB411062E
:1066600090029902667FB420069002A302667FE53D
:106670005375F06484C0F0D0E01264B89002AC228C
:1066800020150122758205126B52600F75F00212FF
:1066900005DBD5F0FAD582EF126B5474757882124F
:1066A00007135015207414D274126B547518C075EA
:1066B0001900751A0D1216FB22C2741201622035E0
:1066C0000420362E227880E6543FF5F07978E36591
:1066D000F0701C09E3787F667015203711D23712ED
:1066E0006B547518C0751900751A0D1216FB2230FF
:1066F000362A7880E6543FF5F0797AE365F0701C2D
:1067000009E3787F667015203711D237126B547504
:1067100018C0751900751A0D1216FB22C23722C255
:10672000AC1217396024F51888191212B853590F92
:10673000535A0FC2AFE55AB55906D2AFD3026748D4
:10674000055A535A0FD2AFC380D7D2AC227E007FF6
:106750007890000075F000E49325F0F5F0A3C3E510
:10676000829EE5839F40F0E5F0700122E5F0C0E0F5
:10677000E5831264B9E5821264B9D0E01264B9C24B
:10678000ADC2ACD21712067520B7FA75F0C8120563
:10679000DBD5F0FA30B7FD75F0C81205DBD5F0FA9D
:1067A000126E9E2275F064120B9E20E51230E30FEC
:1067B000221205F3B2B51205F3B2B5D5F0F322C239
:1067C000AFB2B51205F3B2B51205F3D5F0D9C2A038
:1067D00075F0321267B1D2A075F0321267B1C2A063
:1067E00075F0321267B1D2A075F0321267B175F050
:1067F000961267B180D822300A3C74007892120752
:106800002240337F087E0074787882120713CE13FB
:10681000CE05E0DFF420180E740078A21207225093
:1068200005EE655560108E558E537518C0751904A8
:1068300085531A1216FB22C2AF75181075190FF581
:106840001A1216FBD2AF22300A0C206909740178A3
:106850009212072250012274777882120713E49271
:10686000E0C0E074767882120713D0E033FE20187F
:106870000E740178A21207225005EE655660D78E7D
:1068800056EE20E10630E0440268EE30E022A26BD2
:10689000726A50C2C26BC26AC2AF754D00754E01BA
:1068A000D2AFC227757700D2A774F812683780A6D6
:1068B000D26BC26AC2AF754D00754E01D2AFC2270E
:1068C000757700D2A774F7126837808A206A87D25A
:1068D0006AC26BC2AF754D00754E01D2AFC227754B
:1068E0007700D2A7D26874F6126837026856A227DA
:1068F000826A40F7D26AC26BC20C12279574F512F5
:106900006837026856C082C083D083D08222222298
:10691000C2A075F0141205DBD5F0FAD2A075F01400
:106920001205DBD5F0FA22C2A075F03C1205DBD5CA
:10693000F0FAD2A075F0141205DBD5F0FA22126934
:106940001012691012692712691075F0641205DBC4
:10695000D5F0FA2212692712691012691012691013
:1069600075F0641205DBD5F0FA22305009C2A3C2DB
:1069700063D2A4C26422D2A3C263C2A4C26422228C
:10698000300AFCA26C926E300A1CC0E078D4E2603F
:1069900013C3335005D0E00269BC12062750F6D06D
:1069A000E00269A6D0E0D26C201803206ED17518E1
:1069B000C0751900751A0F1216FB80C3C26C20181F
:1069C00003306EBB7518C0751900751A101216FBCE
:1069D000A26D926E300A1CC0E078DCE26013C33313
:1069E0005005D0E0026A0A12062750F6D0E002698C
:1069F000F3D0E0D26D201803206E237518C07519EE
:106A000000751A181216FB026A1EC26D2018033098
:106A10006E0C7518C0751900751A191216FB22C272
:106A2000B675380074031253BCE51E1253BCE51F43
:106A30001253BC744E1253BC74081253BC7401122E
:106A400053BC74061253BC7854E2F5F0E5F01253CF
:106A5000BC08E2F5F0E5F01253BC7856E2F5F0E53B
:106A6000F01253BC08E2F5F0E5F01253BC244AF8EA
:106A7000E27858E2547FF5F0784CE2C36001D3E548
:106A8000F092E7F5F0E5F01253BC75F000E5F01276
:106A900053BCE5381253BC3099FD22C2B61274893A
:106AA00012741875380074031253BCE51E1253BCDF
:106AB000E51F1253BC744E1253BC740C1253BC74B9
:106AC000001253BC740A1253BCC082C083A3A3A398
:106AD000E49375F064A4C0E0E5F01253BCD0E0127A
:106AE00053BCA3A3A3A3E49375F064A4C0E0E5F0B2
:106AF0001253BCD0E01253BCD083D082E493125323
:106B0000BCA3E4931253BCA3A3A3E4931253BCA36A
:106B1000E4931253BCE58D1253BCE58B1253BCE5D4
:106B2000381253BC3099FD22120A95C28474541253
:106B30000AAFE4120A6F120A82F5F06448255F3347
:106B4000F55FE5F02560B2E003F560D9E9D2842273
:106B50002222E4227583DD75F010753003858331C0
:106B6000753200C083C0F0120954120E6DD0F0D0FF
:106B7000830583D5F0E47533FF7534FF126B5175CF
:106B8000780075790022026BB9C082C083758205D6
:106B9000C082126B52D082601CC2A075F00F120529
:106BA000DBD5F0FAD2A075F0051205DBD5F0FAD5E9
:106BB00082DE126B54D083D082E5822400C0E0E5EF
:106BC0008334DDF8D0E0C322C082C0837401F9743D
:106BD0007CF8753003858331858232120A4A787CCD
:106BE000B6020CE57924FFF579E57834FFF578D025
:106BF00083D08222126B89C082C083F5828883127F
:106C00006BC8787C76007401F9747CF87530038564
:106C1000833185823212099FD083D082126B512238
:106C2000126B89C082C083F5828883C082C083745E
:106C300001F9747CF8753003858331858232120A3C
:106C40004A787CB60209D083D082D083D08222E5F4
:106C5000792401F57950020578D083D082787C764A
:106C6000027401F9747CF8753003858331858232B2
:106C700012099FD083D082126B5122126B89126B42
:106C800089C082C083F5828883126BC8787C7601C4
:106C90007401F9747CF87530038583318582321272
:106CA000099FD083D082126B5122126B89C082C09F
:106CB00083F5828883126BC8787C76037401F9743B
:106CC0007CF875300385833185823212099FD08329
:106CD000D082126B5122126B868003126B89C082A4
:106CE000C083F58288837401F9747CF8753003855C
:106CF0008331858232120A4A787CE6B40102800C24
:106D0000B402028007B4030280027400D083D082F0
:106D100022120A95C2847454120AAFE4120A6F1246
:106D20000A82B40205755F018002D9F3D28422750C
:106D30005F007583DD75F00F753003858331753223
:106D400000C083C0F0120954120AC5120954790018
:106D5000126D11D0F0D0830583E55F7026D5F0D891
:106D6000753003858331753200120954120AC51239
:106D7000095479A0126D117533FF7534FFE55F700A
:106D800002D322C322C28C758A45758C5DD28CB227
:106D90000020000132C0D0C0E0C0F075D008D26140
:106DA000121751126E7F051DE51D20E00C20E10930
:106DB000301716E51D541F6034201704E54C60029F
:106DC000B2B5D0F0D0E0D0D032206605A227B39281
:106DD000A2E51D30E203123853E51D541F7011D295
:106DE00062B5484DB54A5CB56464B57065B54B6A2B
:106DF000E4B54C4BB54972B54673B54F77B5777866
:106E0000E54E454D6029E54E2401F54E5002054DF5
:106E1000454D701BC20B206916206A13C2AF754D19
:106E200000754E01D2AFC227757700D2A7D2688015
:106E300088D548B0C20B754AB4D254D25780A51534
:106E40004C80B1D54AA1C252C253C2548099156434
:106E50008098D57098757A008093D54B93754703C9
:106E60003017030260BD026DE71549808AD5468A56
:106E7000D25B8086154F8085D57785C2A78081E556
:106E80001DA2E330630292A330660292A230650233
:106E900092A122C2B6205C02D2B6126E9E3275C892
:106EA00000C2ADC2AC75CBFF75CA9875CDFF75CC6D
:106EB00098759853C298C299D2ACC2BC75C8347543
:106EC00099062275C800C2ACC2AD75980075CC2B6E
:106ED00075CDEBD2AD75C8042275C800C2ACC2AD89
:106EE000759800E58A242BF5CC540F658C24EBF5BE
:106EF000CDD2AD75C80422C2A8C2AAC289C28BC2B3
:106F0000ACC2A9C2AB758F01120BABD217D2A0C213
:106F1000AF754D00754E01D2AFC227757700D2A76D
:106F2000E4F53C7860F2788275F010F2D5F0FCC29E
:106F300069C26AC26BC26CC26D753E0F75400F7537
:106F40001D04C251C252C253C254754A01754B004E
:106F5000C257D261757400C237C219C21AD25BC25D
:106F60005C754610E4F542F543F544F535F5371206
:106F700024F3751E00751F80E4F548F551F550F5B2
:106F800059F55AF53FC224C225C226C22C7437785F
:106F900065F27866F27867F274377868F2D2207515
:106FA000470375490178A87A0576FF08DAFB757BF7
:106FB000007820E47A07F208DAFCC2117553FF85E5
:106FC0005355C212C20AC209C23875641E756600E2
:106FD000C273C20FC210C20BC20CC20DC26FC2700C
:106FE00075620075610075F00A784AE4F208D5F020
:106FF000FB7954E4F309F37956F309F37858E4F292
:107000001219C1754CFAB2B57533FF7534FFD274DD
:10701000756F00782F740AF2D206127468757A00C0
:1070200075700175731AC201C204C20575770075C7
:107030007800757900758901758A3E758C5DC2B9D5
:10704000D2A9D28CD2B6126E9ED2AFD293C2B4D293
:10705000B2B2B522C21775520375F0031205DBD523
:10706000F0FAC26FC270123D5A75520375F00312E6
:1070700005DBD5F0FAC26FC270123BE5C2AF121841
:10708000CE020000200505200102C322121A5C1264
:10709000721AD322C2AF754CFAB2B51205F3B2B56B
:1070A0001205F3B2B5D2A07581CD75D000126EF77E
:1070B00012690512674D126B541223C8754CFA12EF
:1070C00011B6127084755203123EDB1206C2751897
:1070D00080751904751A7D1216FBD218300A0F122A
:1070E000104E1267F7126847126680126980D2B795
:1070F000D2AFC217C21800000020B7091205F32052
:10710000B7030223E2300A1530380312104E300A5A
:107110000C1267F7126847126680126980E5666094
:1071200003D5660E12758D304603123FCC1265DB17
:10713000800CD2A3C263C2A1D265D2A4C264E564AA
:10714000700630380312671FC266D2A1C265126989
:107150006AC26FC270D268786BE2600D24FD40098C
:107160007576021240B2127084786CE2600D24FDD4
:1071700040097576031240B212708430470620A889
:107180000312334B122723205E08205D05205F0287
:10719000801A3030093053061269050271A4124773
:1071A00071127084782FE215E0F27008782F741451
:1071B000F20270EE02710E00207521C0D0C0E0E82E
:1071C000C0E0C0F0E54F7003857371754F08D27849
:1071D000127292D0F0D0E0F8D0E0D0D0C289322044
:1071E0007526C0D0C0E0E8C0E0C0F0E54F70038570
:1071F0007371754F08C278127292308502D204D032
:10720000F0D0E0F8D0E0D0D0C28B32C2A8C2AAC27F
:1072100093C2B4C0E01205DBD0E0C293C2B4C2890D
:10722000C28BD2B2D2B3C275754F00857371C204DE
:10723000C2B8D288D2A8C2BAD28AD2AA22C2A8C25E
:10724000AAC289C28B22E573141475F00884F5F084
:10725000C0F07836E230E002B27630E102B2763049
:10726000E202B27630E302B27608D5F0E7D0F0E27F
:1072700030E002B27730E102B27730E202B277302A
:10728000E302B27708D5F0E7207605307702C32213
:10729000D322E571B57307A27892760272DCB4014D
:1072A00007A27892770272DCC3E5731495714032BD
:1072B00075F004842436F8E205F0D5F006A2789241
:1072C000E38016D5F006A27892E2800DD5F006A2F2
:1072D0007892E18004A27892E0540FF2D57102D244
:1072E0007522857371D2752275493212720B306125
:1072F00005C26112073CE54960113075F1E5717016
:107300000A12723D1272464002C32212723DD3220B
:10731000094300A00954009F0966009E0977009D5B
:107320000989009C099B009B09AD009A09BF00993F
:1073300009D2009809E4009709F700960A0A009517
:107340000A1D00940A3000930A4300920A570091E4
:107350000A6B00900A7F008F0A93008E0AA7008DA7
:107360000ABB008C0AD1008B0AE7008A0AFE00895A
:107370000B1400880B2B00870B4300860B5C0085E9
:107380000B7500840B8E00830BA700820BC100815C
:107390000BDB00800BF6007F0C10007E0C2B007DB9
:1073A0000C47007C0C64007B0C81007A0C9E0079F9
:1073B0000CBB00780CDB00770CFB00760D1B007516
:1073C0000D3B00740D5B00730D7D00720D9F00710D
:1073D0000DC200700DE4006F0E07006E0E2C006DE4
:1073E0000E51006C0E76006B0E9B006A0EC1006998
:1073F0000EE900680F1100670F3900660F61006524
:107400000F8900640FB300630FDE00621009006192
:1074100010340060105F005F7F42907310E493A30C
:10742000F5F0E493A3C3958BE5F0958D5015A3A3D8
:10743000DFEBE58224FFF582E58334FFF583E493F7
:1074400014800BA3E493BF42059073108010C0E03A
:10745000E58224F9F582E58334FFF583D0E02290BC
:107460000073E0A28733F0229000747400F0900063
:10747000737455F090007574FFF09000777405F008
:107480009000767412F0D28122D286A2A4C0D0D20B
:10749000A475F000D5F0FDD5F0FDC28E53890F43E1
:1074A0008910758B00758D00C28FC2AFC2A4D28EB9
:1074B000208603308FFAC28E308F06758BFF758D54
:1074C000FFD2AFD0D092A422F024FE40053081023A
:1074D000C28122900077E0D5E0EE7442F012748908
:1074E000D281E58B2499E58D34F24014E58B24E1BB
:1074F000E58D34F3400EE58B24E0E58D34FC400847
:1075000074158006741180027412FE900076E06E8D
:107510006010EEF020030B7518C07519008E1A125A
:1075200016FB2212745F6036046033900075E02011
:10753000E010D2E0F0900074E070047405F022E4F2
:10754000F022900074E0602914F07025200222756A
:1075500018C0751900751A141216FB027571900087
:1075600075E030E00DC2E0F0900074E070D1743C42
:10757000F022900074E060F914F070F52002F275CA
:1075800018C0751900751A131216FB80E41274D313
:10759000127523220000000000000000000000001F
:1075A00000000000000000000000000000000000DB
:1075B00000000000000000000000000000000000CB
:1075C00000000000000000000000000000000000BB
:1075D00000000000000000000000000000000000AB
:1077C0000000000000000000000000000000505217
:1077D000343032207665722E3132352E32204864B4
:1077E000773A482034303030752031342D31312D06
:1077F00030342031323A343920204352433D003F67
:00000001FF
:0300000306028072
